:0200000480007A
:10000000B72F0000938F0F8073900F306F00400365
:100010001300000013000000130000001300000094
:100020001300000013000000130000001300000084
:100030001300000013000000130000001300000074
:100040009702000093824211739052309300000097
:10005000130100009301000013020000930200004E
:100060001303000093030000130400009304000036
:10007000130500009305000013060000930600001E
:100080001307000093070000130800009308000006
:100090001309000093090000130A0000930A0000EE
:1000A000130B0000930B0000130C0000930C0000D6
:1000B000130D0000930D0000130E0000930E0000BE
:1000C000130F0000930F000097110200938141BEAF
:1000D000170502001305053F9795030093854570AA
:1000E00013060000EF00001A170502001305853BF8
:1000F000970502009385853B13060000EF008018EA
:1001000017A503001305056E97B503009385456D8C
:1001100037B6ABAB1306B6BAEF00C01617B1030083
:100120001301416CEF7040399392120093D2120088
:100130009382D2FF638A02008322010013014100EF
:100140006F0000177300203083220100130141006B
:10015000730020301301C1FF23205100F32220340B
:10016000E3C402FC8322010013014100130141F8A2
:1001700023221100232421002326310023284100BB
:10018000232A5100232C6100232E71002320810299
:10019000232291022324A1022326B1022328C10293
:1001A000232AD102232CE102232EF1022320010570
:1001B0002322110523242105232631052328410567
:1001C000232A5105232C6105232E71052320810745
:1001D000232291072324A1072326B1072328C1073F
:1001E000232AD107232CE107232EF107732520347E
:1001F000F3251034130601006F000000731015344E
:1002000083204100032181008321C10003220101D9
:1002100083224101032381018323C10103240102BD
:1002200083244102032581028325C10203260103A1
:1002300083264103032781038327C1030328010485
:1002400083284104032981048329C104032A010569
:10025000832A4105032B8105832BC105032C01064D
:10026000832C4106032D8106832DC106032E010731
:10027000832E4107032F8107832FC1071301C10775
:10028000730020302320C5006376B50013054500B8
:100290006FF05FFF678000000000000000000000BA
:1002A000000000000000000000000000000000004E
:1002B000130101F8232011002322210023243100FF
:1002C0002326410023285100232A6100232C71009A
:1002D000232E8100232091022322A1022324B10294
:1002E0002326C1022328D102232AE102232CF10272
:1002F000232E010323201105232221052324310568
:100300002326410523285105232A6105232C710545
:10031000232E8105232091072322A1072324B1073F
:100320002326C1072328D107232AE107232CF1071D
:100330009702020083A2021723A02200F3221034A6
:10034000232E5106EF00804617010200032181157C
:10035000032101008322C10773901234B7220000E9
:100360009382028873A00230832001000322C1001F
:100370008322010103234101832381010324C1015D
:100380008324010203254102832581020326C10241
:100390008326010303274103832781030328C10325
:1003A000832801040329410483298104032AC10409
:1003B000832A0105032B4105832B8105032CC105ED
:1003C000832C0106032D4106832D8106032EC106D1
:1003D000832E0107032F4107832F81071301010893
:1003E00073002030970202009382C20D23A01200F6
:1003F00023A2220023A4320023A6420023A85200F5
:1004000023AA620023AC720023AE820023A09202D2
:1004100023A2A20223A4B20223A6C20223A8D202CC
:1004200023AAE20223ACF20223AE020323A01205A8
:1004300023A2220523A4320523A6420523A85205A0
:1004400023AA620523AC720523AE820523A092077E
:1004500023A2A20723A4B20723A6C20723A8D20778
:1004600023AAE20723ACF207EF6010731701020022
:1004700003214103032101008322C1077390123439
:10048000B72200009382028873A00230832001000B
:100490000322C1008322010103234101832381013F
:1004A0000324C10183240102032541028325810223
:1004B0000326C10283260103032741038327810307
:1004C0000328C103832801040329410483298104EB
:1004D000032AC104832A0105032B4105832B8105CF
:1004E000032CC105832C0106032D4106832D8106B3
:1004F000032EC106832E0107032F4107832F810797
:10050000130101087300203097020200938282FBDE
:1005100083A0020003A1420083A1820003A2C200C3
:1005200083A2020103A3420183A3820103A4C201A7
:1005300083A4020203A5420283A5820203A6C2028B
:1005400083A6020303A7420383A7820303A8C2036F
:1005500083A8020403A9420483A9820403AAC20453
:1005600083AA020503AB420583AB820503ACC20537
:1005700083AC020603AD420683AD820603AEC2061B
:1005800083AE020703AFC20983AF82076780000012
:1005900073700430130101F823201100232221007D
:1005A000232431002326410023285100232A6100FF
:1005B000232C7100232E8100232091022322A102EB
:1005C0002324B1022326C1022328D102232AE102D7
:1005D000232CF102232E01032320110523222105C0
:1005E000232431052326410523285105232A6105AB
:1005F000232C7105232E8105232091072322A10797
:100600002324B1072326C1072328D107232AE10782
:10061000232CF1079702020083A2C2E823A0220044
:10062000232E1106EF20D05817010200032181E785
:10063000032101008322C10773901234B722000006
:100640009382028873A00230832001000322C1003C
:100650008322010103234101832381010324C1017A
:100660008324010203254102832581020326C1025E
:100670008326010303274103832781030328C10342
:10068000832801040329410483298104032AC10426
:10069000832A0105032B4105832B8105032CC1050A
:1006A000832C0106032D4106832D8106032EC106EE
:1006B000832E0107032F4107832F810713010108B0
:1006C0007300203097070200938787DE03A7070097
:1006D0009307F0FF6306F700737004306F000000AB
:1006E000737004306F000000130101FF2326A10086
:1006F0008327C100739047301300000013010101EC
:1007000067800000130101FFF32740302326F1002A
:1007100073F043308327C1001385070013010101E3
:1007200067800000130101FF2326A1002324B100EC
:100730002322C1008327C1009387C7FF2326F1002E
:10074000032781008327C10023A0E7008327C1007E
:10075000938787FA2326F100032741008327C100EE
:1007600023A0E7008327C100938787FE2326F1009B
:1007700093870100138707008327C10023A0E700A8
:100780008327C100938747FF2326F1001707000046
:10079000130787F38327C10023A0E7008327C10045
:1007A000138507001301010167800000130101FF99
:1007B00023261100EF60D033EF20101693070500B9
:1007C00063840700EF20D03E130000008320C100A7
:1007D0001301010167800000130101FF2326A1001E
:1007E0008327C100138787008327C10023A2E70066
:1007F0008327C1001307F0FF23A4E7008327C1006C
:10080000138787008327C10023A6E7008327C10041
:10081000138787008327C10023A8E7008327C1002F
:1008200023A00700130000001301010167800000EE
:10083000130101FF2326A1008327C10023A807007D
:10084000130000001301010167800000130101FE85
:100850002326A1002324B1008327C10083A74700DA
:10086000232EF100832781000327C10123A2E70083
:100870008327C10103A787008327810023A4E70002
:100880008327C10183A787000327810023A2E700F4
:100890008327C1010327810023A4E7008327810068
:1008A0000327C10023A8E7008327C10083A707000F
:1008B000138717008327C10023A0E700130000005F
:1008C0001301010267800000130101FE2326A1002D
:1008D0002324B1008327810083A70700232CF10084
:1008E000032781019307F0FF631AF7008327C100F4
:1008F00083A70701232EF1006F0040038327C10067
:1009000093878700232EF1006F0000018327C10128
:1009100083A74700232EF1008327C10183A7470047
:1009200083A7070003278101E372F7FE8327C10134
:1009300003A747008327810023A2E70083278100C4
:1009400083A747000327810023A4E70083278100B2
:100950000327C10123A4E7008327C10103278100E6
:1009600023A2E700832781000327C10023A8E70013
:100970008327C10083A70700138717008327C100BF
:1009800023A0E700130000001301010267800000AC
:10099000130101FE2326A1008327C10083A70701BD
:1009A000232EF1008327C10083A747000327C1003E
:1009B0000327870023A4E7008327C10083A78700BC
:1009C0000327C1000327470023A2E7008327C101B3
:1009D00083A747000327C100631AF7008327C100DC
:1009E00003A787008327C10123A2E7008327C10053
:1009F00023A807008327C10183A707001387F7FFF8
:100A00008327C10123A0E7008327C10183A7070033
:100A1000138507001301010267800000130101FD27
:100A200023261102232481022326A1002324B100BE
:100A30008327C100232EF1008327C101639607009D
:100A4000737004306F000000EF3010418327C10144
:100A500003A407008327C10103A7C7038327C1019C
:100A600083A707049385070013050700EF90C01FB5
:100A7000930705003307F4008327C10123A2E70091
:100A80008327C10123AC07028327C10103A7070005
:100A90008327C10123A4E7008327C10103A4070022
:100AA0008327C10183A7C7031387F7FF8327C101EA
:100AB00083A707049385070013050700EF90C01A6A
:100AC000930705003307F4008327C10123A6E7003D
:100AD0008327C1011307F0FF23A2E7048327C10185
:100AE0001307F0FF23A4E70483278100639A07021A
:100AF0008327C10183A70701638407048327C101FA
:100B00009387070113850700EF20504C130705005A
:100B1000930710006316F702EFF09FA76F004002E3
:100B20008327C1019387070113850700EFF0DFCA10
:100B30008327C1019387470213850700EFF0DFC9C0
:100B4000EF30903593071000138507008320C10212
:100B5000032481021301010367800000130101FDDA
:100B6000232611022326A1002324B10093070600A7
:100B7000A303F100232C01008327C1006396070023
:100B8000737004306F0000008327810063960700B4
:100B9000232E01006F00C001832581000325C100C1
:100BA000EF90800C9307050093871700232EF10028
:100BB0008327C1019387470513850700EF50006E17
:100BC000232AA1008327410163820706832781002E
:100BD000639A0700832741010327410123A0E7000F
:100BE0006F00400183274101138747058327410197
:100BF00023A0E700832741010327C10023AEE702BA
:100C0000832741010327810023A0E70493051000F7
:100C100003254101EFF09FE0832741010347710065
:100C20002388E70483274101232CF10083278101D6
:100C300063960700737004306F0000008327810102
:100C4000138507008320C1021301010367800000A0
:100C5000130101FD2326110293070500A307F100EC
:100C600013054005EF508063232EA1008327C101A7
:100C7000638C07088327C10123A207008327C101D2
:100C800023A007008327C10123A407008327C101F4
:100C900023A607008327C10123AC07028327C101D4
:100CA0001307100023AEE7028327C10123A0070426
:100CB0008327C1011307F0FF23A2E7048327C101A3
:100CC0001307F0FF23A4E7048327C1010347F100C2
:100CD0002388E7048327C101938707011385070051
:100CE000EFF09FAF8327C101938747021385070069
:100CF000EFF09FAE9306000013060000930500007E
:100D00000325C101EF00001E8327C10113850700E1
:100D10008320C1021301010367800000130101FD5C
:100D200023261102232481022326A1008327C10048
:100D3000232CF10083278101639607007370043030
:100D40006F0000008327810103A44700EF3000609B
:100D5000930705006312F4048327810183A7C7006A
:100D60001387F7FF8327810123A6E70083278101EB
:100D700083A7C700639C07009306000013060000CA
:100D80009305000003258101EF00C01593071000B3
:100D9000232EF1006F008000232E01008327C10164
:100DA000138507008320C10203248102130101037C
:100DB00067800000130101FD232611022324810214
:100DC0002326A1002324B1008327C100232CF10096
:100DD0008327810163960700737004306F00000061
:100DE0008327810103A44700EF3040569307050095
:100DF0006312F4028327810183A7C70013871700BA
:100E00008327810123A6E70093071000232EF1001A
:100E10006F00C003930600000326810093050000C5
:100E200003258101EF00C058232EA1000327C10133
:100E300093071000631CF7008327810183A7C70075
:100E4000138717008327810123A6E7008327C101A9
:100E5000138507008320C1020324810213010103CB
:100E600067800000130101FD232611022326A10043
:100E70002324B1008327C1006396070073700430F8
:100E80006F000000032781008327C10063F6E7009D
:100E9000737004306F0000001306200093050000FB
:100EA0000325C100EFF09FCB232EA1008327C101B2
:100EB000638807008327C1010327810023ACE70271
:100EC0008327C10163960700737004306F00000030
:100ED0008327C101138507008320C1021301010389
:100EE00067800000130101FC232E11022326A100BC
:100EF0002324B1002322C1002320D1002326010294
:100F00008327C1002324F10283278102639607000F
:100F1000737004306F00000083278100639807001E
:100F20008327810283A707046396070093071000B5
:100F30006F00800093070000639607007370043011
:100F40006F0000000327010093072000631AF700D9
:100F50008327810203A7C703930710006316F700D6
:100F6000930710006F00800093070000639607004E
:100F7000737004306F000000EF30803F930705006E
:100F800063960700832741006396070093071000CC
:100F90006F008000930700006396070073700430B1
:100FA0006F000000EF30406B8327810203A78703A7
:100FB0008327810283A7C7036368F7000327010023
:100FC000930720006310F7060326010083258100A4
:100FD00003258102EF00101C2322A1028327810236
:100FE00083A747026384070283278102938747020E
:100FF00013850700EF20807D13070500930710007D
:10100000631CF700EFF0CFD86F0000018327410287
:1010100063840700EFF0CFD7EF300068930710002C
:101020006F00400F8327410063980700EF30C066D0
:10103000930700006F00000E8327C102639C070026
:101040009307C10113850700EF20501D930710007F
:101050002326F102EF304064EF10D049EF30C05F3B
:101060008327810203A747049307F0FF6316F70065
:101070008327810223A207048327810203A7870411
:101080009307F0FF6316F7008327810223A4070468
:10109000EF308060130741009307C10193050700FB
:1010A00013850700EF20501C93070500639C07047D
:1010B00003258102EF00504693070500638C070269
:1010C00083278102938707010327410093050700C7
:1010D00013850700EF20004A03258102EF00902CC2
:1010E000EF10904393070500E39E07EAEFF04FCA25
:1010F0006FF05FEB03258102EF00D02AEF10D041A3
:101100006FF05FEA03258102EF00D029EF10D04095
:1011100093070000138507008320C1031301010416
:1011200067800000130101FD232611022326A10080
:101130002324B1002322C1002320D1008327C10032
:10114000232CF1008327810163960700737004301C
:101150006F000000832781006398070083278101C7
:1011600083A7070463960700930710006F008000B1
:101170009307000063960700737004306F0000004F
:101180000327010093072000631AF70083278101DA
:1011900003A7C703930710006316F7009307100017
:1011A0006F0080009307000063960700737004309F
:1011B0006F000000EFF00FD593070500232AF10020
:1011C0008327810103A787038327810183A7C7039F
:1011D0006368F70003270100930720006310F708F6
:1011E000032601008325810003258101EF00807A19
:1011F0008327810103A787049307F0FF6310F70497
:101200008327810183A74702638407048327810121
:101210009387470213850700EF20405B9307050083
:101220006388070283274100638407028327410004
:101230001307100023A0E7006F00800183278101BE
:1012400083A78704138717008327810123A4E7045A
:1012500093071000232EF1006F008000232E010061
:101260008327410113850700EFF00FC88327C101D1
:10127000138507008320C10213010103678000006A
:10128000130101FD232611022326A1002324B1000E
:101290008327C100232CF100832781016396070077
:1012A000737004306F0000008327810183A7070457
:1012B00063860700737004306F000000832781018C
:1012C00083A70700639807008327810183A747004E
:1012D00063960700930710006F00800093070000DB
:1012E00063960700737004306F000000EFF08FC149
:1012F00093070500232AF1008327810103A78703B1
:101300008327810183A7C7036372F70883278101BD
:1013100083A78703138717008327810123ACE70284
:101320008327810103A787049307F0FF6310F70465
:101330008327810183A747026384070483278101F0
:101340009387470213850700EF2040489307050065
:101350006388070283278100638407028327810053
:101360001307100023A0E7006F008001832781018D
:1013700083A78704138717008327810123A4E70429
:1013800093071000232EF1006F008000232E010030
:101390008327410113850700EFF00FB58327C101B3
:1013A000138507008320C102130101036780000039
:1013B000130101FC232E11022326A1002324B100D6
:1013C0002322C1002320D100232601028327C1004C
:1013D0002324F1028327810263960700737004308F
:1013E0006F00000083278100639807008327810234
:1013F00083A7070463960700930710006F0080001F
:101400009307000063960700737004306F000000BC
:10141000EF201076930705006396070083274100AD
:1014200063960700930710006F0080009307000089
:1014300063960700737004306F000000EF30C02126
:101440008327810283A787036382070C8327810296
:1014500083A7C7002322F10283258100032581028F
:10146000EF00806B832701006392070683278102C8
:1014700083A787031387F7FF8327810223ACE70243
:101480008327810283A70700639A0700EF30802B30
:10149000130705008327810223A2E7008327810227
:1014A00083A70701638E07048327810293870701BF
:1014B00013850700EF208031130705009307100004
:1014C0006310F704EFF0CF8C6F0080038327810255
:1014D0000327410223A6E7008327810283A747024F
:1014E00063800702832781029387470213850700E1
:1014F000EF20C02D9307050063840700EFF04F89AC
:10150000EF308019930710006F008011832741008E
:1015100063980700EF304018930700006F004010F9
:101520008327C102639C07009307C101138507004D
:10153000EF20C04E930710002326F102EF30C015B4
:10154000EF10407BEF3040118327810203A747044F
:101550009307F0FF6316F7008327810223A2070495
:101560008327810203A787049307F0FF6316F70020
:101570008327810223A40704EF30001213074100E0
:101580009307C1019305070013850700EF20C04DA5
:1015900093070500639E070603258102EF00406F55
:1015A00093070500638E07048327810283A7070042
:1015B000639E0700EF30400A8327810283A747001C
:1015C00013850700EF20D05FEF30000D83278102E5
:1015D00093874702032741009305070013850700FF
:1015E000EF10507903258102EF00C05BEF10C0724D
:1015F00093070500E39407E4EFE09FF96FF01FE421
:1016000003258102EF00005AEF1000716FF01FE315
:1016100003258102EF000059EF10007093070000CE
:10162000138507008320C1031301010467800000B4
:10163000130101FD232611022326A1002324B1005A
:101640002322C1008327C100232CF10083278101BD
:1016500063960700737004306F00000083278100D9
:10166000639807008327810183A707046396070017
:10167000930710006F008000930700006396070037
:10168000737004306F000000EFF0CF879307050000
:10169000232AF1008327810183A787036388070832
:1016A0008325810003258101EF0000478327810105
:1016B00083A787031387F7FF8327810123ACE70202
:1016C0008327810103A747049307F0FF6310F70402
:1016D0008327810183A7070163840704832781018E
:1016E0009387070113850700EF20400E930705003D
:1016F0006388070283274100638407028327410030
:101700001307100023A0E7006F00800183278101E9
:1017100083A74704138717008327810123A2E704C7
:1017200093071000232EF1006F008000232E01008C
:101730008327410113850700EFE01FFB8327C101C9
:10174000138507008320C102130101036780000095
:10175000130101FD232611022326A1002324B10039
:101760008327C100232CF1008327810163960700A2
:10177000737004306F0000008327810063980700B6
:101780008327810183A7070463960700930710004E
:101790006F008000930700006396070073700430A9
:1017A0006F0000008327810183A707046396070069
:1017B000737004306F000000EFE0DFF49307050062
:1017C000232AF1008327810183A78703638A070205
:1017D0008327810183A7C7002328F1008325810087
:1017E00003258101EF004033832781010327010195
:1017F00023A6E70093071000232EF1006F0080005E
:10180000232E01008327410113850700EFE0DFED60
:101810008327C101138507008320C102130101033F
:1018200067800000130101FD232611022326A10079
:101830008327C10063960700737004306F000000B7
:10184000EF2090618327C10083A78703232EF10037
:10185000EF2090648327C101138507008320C10214
:101860001301010367800000130101FD232611020B
:101870002326A1008327C100232EF1008327C10165
:1018800063960700737004306F000000EF20D05C97
:101890008327C10103A7C7038327C10183A7870348
:1018A000B307F740232CF100EF20105F832781015D
:1018B000138507008320C102130101036780000024
:1018C000130101FE2326A1008327C10063960700B0
:1018D000737004306F0000008327C10083A7870363
:1018E000232EF1008327C101138507001301010294
:1018F00067800000130101FD232611022326A100A9
:101900008327C100232EF1008327C10163960700BE
:10191000737004306F0000000325C101EF004052D6
:101920000325C101EF405037130000008320C1029E
:101930001301010367800000130101FF2326A100AA
:101940008327C10083A7C704138507001301010182
:1019500067800000130101FF2326A1002324B100AA
:101960008327C1000327810023A6E704130000009A
:101970001301010167800000130101FF2326A1006C
:101980008327C10083C707051385070013010101E1
:1019900067800000130101FD232611022326A10008
:1019A0002324B1002322C100232E01008327C1007C
:1019B00083A70704639807028327C10083A7070052
:1019C000639807128327C10083A747001385070088
:1019D000EF20D034232EA1008327C10023A20700CB
:1019E0006F00001183274100639407068327C1001D
:1019F00003A787008327C10083A707041386070076
:101A00008325810013050700EF40D03F8327C100E5
:101A100003A787008327C10083A707043307F700C4
:101A20008327C10023A4E7008327C10003A7870001
:101A30008327C10083A74700636CF70A8327C1008F
:101A400003A707008327C10023A4E7006F00400A13
:101A50008327C10003A7C7008327C10083A707040A
:101A6000138607008325810013050700EF40903996
:101A70008327C10003A7C7008327C10083A70704EA
:101A8000B307F0403307F7008327C10023A6E70020
:101A90008327C10003A7C7008327C10083A70700CE
:101AA0006372F7028327C10003A747008327C100A1
:101AB00083A70704B307F0403307F7008327C1006B
:101AC00023A6E70003274100930720006312F702D3
:101AD0008327C10083A78703638C07008327C10086
:101AE00083A787031387F7FF8327C10023ACE7028F
:101AF0008327C10083A78703138717008327C100AB
:101B000023ACE7028327C101138507008320C102AC
:101B10001301010367800000130101FE232E110051
:101B20002326A1002324B1008327C10083A7070433
:101B3000638207068327C10003A7C7008327C1006C
:101B400083A707043307F7008327C10023A6E70014
:101B50008327C10003A7C7008327C10083A74700CD
:101B6000636AF7008327C10003A707008327C1002A
:101B700023A6E7008327C10003A7C7008327C1006E
:101B800083A7070413860700930507000325810038
:101B9000EF405027130000008320C1011301010210
:101BA00067800000130101FE232E11002326A100EF
:101BB000EF20902A6F0000048327C10083A747020B
:101BC000638207048327C1009387470213850700B8
:101BD000EF10D03F9307050063840700EF10D07823
:101BE0008327C10083A787041387F7FF8327C100DA
:101BF00023A4E7048327C10083A78704E34EF0FAF8
:101C00006F008000130000008327C1001307F0FF5E
:101C100023A4E704EF205028EF2010246F000004D5
:101C20008327C10083A70701638207048327C100BC
:101C30009387070113850700EF10503993070500BC
:101C400063840700EF1050728327C10083A7470405
:101C50001387F7FF8327C10023A2E7048327C1006E
:101C600083A74704E34EF0FA6F00800013000000E2
:101C70008327C1001307F0FF23A2E704EF20D02140
:101C8000130000008320C1011301010267800000DE
:101C9000130101FD232611022326A100EF20D01BF2
:101CA0008327C10083A78703639807009307100069
:101CB000232EF1006F008000232E0100EF20D01DA5
:101CC0008327C101138507008320C102130101038B
:101CD00067800000130101FE2326A1008327C100B5
:101CE00063960700737004306F0000008327C10003
:101CF00083A787036398070093071000232EF10042
:101D00006F008000232E01008327C1011385070087
:101D10001301010267800000130101FD2326110257
:101D20002326A100EF2050138327C10003A78703B8
:101D30008327C10083A7C7036318F7009307100028
:101D4000232EF1006F008000232E0100EF20D0141D
:101D50008327C101138507008320C10213010103FA
:101D600067800000130101FE2326A1008327C10024
:101D700063960700737004306F0000008327C10072
:101D800003A787038327C10083A7C7036318F7004E
:101D900093071000232EF1006F008000232E010016
:101DA0008327C1011385070013010102678000002A
:101DB000130101FE2326A1002324B100232E0100DC
:101DC0006F008006178703001307C79D8327C10193
:101DD00093973700B307F70083A7070063900704C2
:101DE000178703001307079C8327C10193973700C8
:101DF000B307F7000327810023A0E700178703003C
:101E00001307479A8327C10193973700B307F70059
:101E10000327C10023A2E7006F00C0018327C1018F
:101E200093871700232EF1000327C1019307700049
:101E3000E3FAE7F8130000001301010267800000D5
:101E4000130101FE2326A100232E01006F00C00410
:101E500017870300130707958327C101939737005E
:101E6000B307F70083A747000327C1006310F702F9
:101E700017870300130707938327C1019397370040
:101E8000B307F70023A007006F00C0018327C1013B
:101E900093871700232EF1000327C10193077000D9
:101EA000E3F8E7FA13000000130101026780000065
:101EB000130101FD232611022326A1002324B100D2
:101EC0002322C1008327C100232EF100EF20C07818
:101ED0008327C10103A747049307F0FF6316F700A8
:101EE0008327C10123A207048327C10103A7870415
:101EF0009307F0FF6316F7008327C10123A40704AB
:101F0000EF2080798327C10183A78703639E0700A1
:101F10008327C1019387470203264100832581005F
:101F200013850700EF10007F0325C101EFF09FC765
:101F3000130000008320C102130101036780000029
:101F4000130101FC232E1102232EA100232CB1002A
:101F50002328D1002326E1002324F10023220101BC
:101F60002320110193070600231BF1008327C101E1
:101F700063960700737004306F0000000327C100F0
:101F80009307900063F6E700737004306F00000061
:101F9000835761018325410013850700EF10D07E30
:101FA0002324A102832781026386071C83278102E1
:101FB00003A7070383566101B70700409387F7FF24
:101FC000B387F60093972700B307F7002322F102A7
:101FD0008327410293F7C7FF2322F102832741029F
:101FE00093F7370063860700737004306F000000BA
:101FF0008357610113870700832601000326C10070
:102000008325810103258102EF1050410326010140
:102010008325C10103254102EFE0CFF0130705003E
:102020008327810223A0E7008327810063880700BC
:10203000832781000327810223A0E700EF20C061EE
:1020400097E701009387476383A70700138717006B
:1020500097E701009387476223A0E70097E7010015
:102060009387474483A707006398070297E7010017
:10207000938747430327810223A0E70097E70100E6
:102080009387875F03A70700930710006312F70485
:10209000EF10904B6F00C00397E701009387875EB6
:1020A00083A707006396070297E701009387873F9E
:1020B00083A7070083A7C7020327C100636AF7004D
:1020C00097E701009387073E0327810223A0E700DB
:1020D00097E701009387075C83A707001387170022
:1020E00097E701009387075B23A0E70097E70100CC
:1020F0009387475A03A707008327810223A4E70495
:102100008327810203A7C70297E7010093874757F8
:1021100083A7070063FCE7008327810203A7C702A8
:1021200097E701009387C75523A0E7008327810223
:1021300003A7C7029307070093972700B387E70019
:102140009397270017E701001307873F3387E700BE
:1021500083278102938747009385070013050700B3
:10216000EFE0CFEE930710002326F102EF20C052DC
:102170006F00C0009307F0FF2326F1020327C1027E
:10218000930710006318F70297E701009387874FC2
:1021900083A707006380070297E7010093878730D2
:1021A00083A7070083A7C7020327C10063F4E700E2
:1021B000EFE00FBE8327C102138507008320C10310
:1021C0001301010467800000130101FD23261102A1
:1021D0002326A100EF2040488327C100639A07000F
:1021E00097E701009387072C83A707006F00800003
:1021F0008327C100232EF1008327C1019387470065
:1022000013850700EFE0CFF88327C10183A787027A
:10221000638A07008327C10193878701138507001D
:10222000EFE00FF78327C1019387470093850700ED
:1022300017E5010013058541EFE04FE197E7010045
:102240009387074283A707001387170097E70100CA
:102250009387074123A0E70097E70100938787430F
:1022600083A707001387170097E70100938787422A
:1022700023A0E700EF20404297E7010093878740C3
:1022800083A707006382070497E7010093878721EC
:1022900083A707000327C1016312F70297E7010034
:1022A0009387C73F83A707006386070073700430D6
:1022B0006F000000EFE0CFAD6F000001EF20C039EC
:1022C000EF208001EF20403D130000008320C10279
:1022D0001301010367800000130101FD2326110291
:1022E0002326A1002324B100232E01008327C1004F
:1022F00063960700737004306F000000832781002D
:1023000063960700737004306F00000097E70100C8
:102310009387C73883A7070063860700737004306C
:102320006F000000EF00101D97E70100938707354D
:1023300083A70700232CF1008327C10083A7070090
:1023400003278100B307F700232AF1008327C10088
:1023500083A70700032781016376F7028327C10063
:1023600083A70700032741016370F7040327410196
:102370008327810163FAE70293071000232EF100FF
:102380006F0080028327C10083A707000327410154
:102390006368F700032741018327810163F6E700A3
:1023A00093071000232EF1008327C100032741016A
:1023B00023A0E7008327C1016382070297E701009A
:1023C0009387470E83A7070093874700138507006D
:1023D000EFE00FDC03254101EF10502FEF00D01389
:1023E0002328A1008327010163940700EFE04F9A9F
:1023F000130000008320C102130101036780000065
:10240000130101FD232611022326A100232E010022
:102410008327C1006380070697E701009387072899
:1024200083A7070063860700737004306F00000005
:10243000EF00500C97E701009387472483A707001C
:102440000327C100B307F700232CF10097E7010031
:102450009387470583A707009387470013850700E5
:10246000EFE00FD303258101EF105026EF00D00AD3
:10247000232EA1008327C10163940700EFE04F9151
:10248000130000008320C1021301010367800000D4
:10249000130101FD232611022326A1008327C10079
:1024A000232CF100832781016396070073700430A9
:1024B0006F00000097E701009387C7FE83A707001E
:1024C000032781016316F700232E01006F00400AE5
:1024D000EF2080188327810183A74701232AF10079
:1024E000EF20801B97E701009387871483A70700DD
:1024F00003274101630CF70097E7010093878713D7
:1025000083A70700032741016318F7009307200002
:10251000232EF1006F00C0050327410197E701005A
:10252000938747146314F7028327810183A78702E7
:102530006398070093073000232EF1006F004003DB
:1025400093072000232EF1006F0080020327410132
:1025500097E701009387870F6318F7009307400000
:10256000232EF1006F00C00093071000232EF1000E
:102570008327C101138507008320C10213010103D2
:1025800067800000130101FD232611022326A1000C
:10259000EF20800C8327C100639A070097E70100B2
:1025A000938747F083A707006F0080008327C1004F
:1025B000232EF1008327C10183A7C702232CF1003A
:1025C000EF20800D83278101138507008320C1023E
:1025D0001301010367800000130101FD232611028E
:1025E0002326A100EFE00F9293070500232EF100B0
:1025F0008327C100639A070097E70100938787EA62
:1026000083A707006F0080008327C100232CF100FF
:102610008327810183A7C702232AF1008327C101F1
:1026200013850700EFE04F8C8327410113850700D6
:102630008320C1021301010367800000130101FD23
:10264000232611022326A1002324B100232E0100FA
:10265000032781009307900063F6E700737004304E
:102660006F000000032781009307900063F6E700E6
:10267000930790002324F100EF10107E8327C10000
:10268000639A070097E701009387C7E183A70700D4
:102690006F0080008327C100232CF1008327810174
:1026A00083A70705232AF10003274101832781001F
:1026B000630EF716032781008327410163FEE702BB
:1026C00097E70100938707DE83A7070003278101AF
:1026D0006302F70497E701009387C7DC83A707002D
:1026E00083A7C702032781006366F70293071000E0
:1026F000232EF1006F00000297E70100938787DA2D
:1027000083A70700032781016316F70093071000D2
:10271000232EF1008327810183A7C7022328F1001C
:102720008327810103A707058327810183A7C702A8
:102730006318F700832781010327810023A6E7029E
:10274000832781010327810023A8E70483278101D0
:1027500083A7870163CC07001307A00083278100AC
:102760003307F7408327810123ACE70083278101EA
:1027700083A64701032701019307070093972700CA
:10278000B387E7009397270017E70100130747DB9C
:10279000B387E7006396F600930710006F00800090
:1027A00093070000638C0706832781019387470006
:1027B00013850700EFE0CF9D8327810103A7C702A0
:1027C00097E701009387C7EB83A7070063FCE70047
:1027D0008327810103A7C70297E70100938747EA90
:1027E00023A0E7008327810103A7C70293070700FF
:1027F00093972700B387E7009397270017E7010017
:10280000130707D43387E7008327810193874700A5
:102810009385070013050700EFE04F830327C101ED
:10282000930710006314F700EFD09FD6EF10D06627
:10283000130000008320C102130101036780000020
:10284000130101FD232611022326A100EF10D06001
:102850008327C100639A070097E70100938787C425
:1028600083A707006F0080008327C100232EF1009B
:102870008327C1019387470013850700EFE04F913D
:102880008327C10183A78702638A07008327C101C9
:102890009387870113850700EFE08F8F8327C1019E
:1028A000938747009385070017E50100130585DB33
:1028B000EFD0DFF9EF10505E97E70100938787BEF6
:1028C00083A707000327C1016314F70697E70100F8
:1028D000938747DB83A707006382070297E701001E
:1028E0009387C7DB83A707006386070073700430F4
:1028F0006F000000EFD0DFC96F00400597E70100CF
:10290000938747D603A7070097E701009387C7D6A9
:1029100083A70700631AF70097E70100938787B83A
:1029200023A007006F008002EF0090286F000002D4
:1029300097E70100938707D583A7070063880700FF
:10294000EF109051EF105019EF10105513000000C8
:102950008320C1021301010367800000130101FEFF
:102960002326A100232E01008327C100232CF10080
:102970008327C10063960700737004306F00000066
:102980008327810103A7470197E70100938787CD3C
:102990006316F700930710006F0080009307000094
:1029A000638E07028327810103A7870297E701004F
:1029B000938787C86304F7028327810183A787026F
:1029C00063960700930710006F00800093070000D4
:1029D0006386070093071000232EF1008327C101AF
:1029E000138507001301010267800000130101FD38
:1029F000232611022326A1008327C100232EF100E4
:102A00008327C10063960700737004306F000000D5
:102A10008327C1016384070C97E70100938787A888
:102A200083A707000327C101630AF70AEF10D0420A
:102A30000325C101EFF09FF2130705009307100073
:102A4000631CF7088327C10193874700138507009C
:102A5000EFD01FF48327C10103A7C70297E7010046
:102A6000938707C283A7070063FCE7008327C101A0
:102A700003A7C70297E70100938787C023A0E70059
:102A80008327C10103A7C702930707009397270075
:102A9000B387E7009397270017E70100130747AABA
:102AA0003387E7008327C101938747009385070099
:102AB00013050700EFD09FD98327C10103A7C702E1
:102AC00097E701009387079E83A7070083A7C702A4
:102AD0006364F700EFD0DFABEF10103C1300000091
:102AE0008320C1021301010367800000130101FD6F
:102AF000232611022326A100232E01008327C100D3
:102B0000232CF1008327C100639607007370043003
:102B10006F000000EFD01FBF93070500232AF100CC
:102B200003258101EFF09FE31307050093071000D1
:102B30006314F70C97E70100938747B683A7070054
:102B40006390070A8327810103A7C70297E7010063
:102B50009387479583A7070083A7C7026366F7009B
:102B600093071000232EF1008327810193874700EC
:102B700013850700EFD0DFE18327810103A7C70298
:102B800097E701009387C7AF83A7070063FCE700BF
:102B90008327810103A7C70297E70100938747AE08
:102BA00023A0E7008327810103A7C702930707003B
:102BB00093972700B387E7009397270017E7010053
:102BC000130707983387E70083278101938747001E
:102BD0009385070013050700EFD05FC76F00C001A2
:102BE00083278101938787019385070017E50100FB
:102BF000130585A4EFD09FC58327410113850700E6
:102C0000EFD09FAE8327C101138507008320C10247
:102C10001301010367800000130101FE232E110040
:102C2000930800001308000093070000130700003A
:102C3000930600001306004097D501009385853C5C
:102C400017150000130505FBEFF08FAF2326A10039
:102C50000327C100930710006316F700EF20C03A66
:102C60002326A1000327C10093071000631EF7026B
:102C70007370043097E70100938707A21307F0FFF2
:102C800023A0E70097E701009387C79F1307100071
:102C900023A0E70097E701009387479E23A0070042
:102CA000EFD04FF46F0040018327C1006396070007
:102CB000737004306F000000130000008320C10116
:102CC0001301010267800000130101FF2326110098
:102CD0007370043097E701009387C79A23A0070019
:102CE000EFD09F82130000008320C1001301010177
:102CF0006780000097E701009387479A83A7070042
:102D00001387170097E701009387479923A0E700EF
:102D10001300000067800000130101FE232E110044
:102D20002326010097E701009387479783A70700B1
:102D300063960700737004306F000000EF10D0112D
:102D400097E701009387879583A707001387F7FF0D
:102D500097E701009387879423A0E70097E7010096
:102D60009387C79383A707006394071697E701002B
:102D70009387879083A70700638C07146F00800CEC
:102D800097E701009387478B83A7C70083A7C700F6
:102D90002324F1008327810093878701138507008F
:102DA000EFD01FBF8327810093874700138507005B
:102DB000EFD01FBE8327810003A7C70297E701005A
:102DC0009387078C83A7070063FCE70083278100B4
:102DD00003A7C70297E701009387878A23A0E7002C
:102DE0008327810003A7C702930707009397270053
:102DF000B387E7009397270017D70100130747749D
:102E00003387E70083278100938747009385070076
:102E100013050700EFD09FA38327810003A7C702F4
:102E200097D701009387076883A7070083A7C70286
:102E3000636AF70097E7010093874785130710003F
:102E400023A0E70097D701009387077F83A7070098
:102E5000E39807F297E701009387078383A70700AA
:102E6000638807046F00C003EF00002B9307050081
:102E7000638A070097E701009387478113071000D3
:102E800023A0E70097E701009387078083A7070047
:102E90001387F7FF97D701009387077F23A0E700E9
:102EA00097D701009387477E83A70700E39E07FA21
:102EB00097D701009387877D03A70700930710002A
:102EC0006318F700930710002326F100EFD04FECB2
:102ED000EF10807C8327C100138507008320C10188
:102EE0001301010267800000130101FE232E11006F
:102EF000EF10807697D701009387477883A7070064
:102F00002326F100EF1040798327C10013850700C5
:102F10008320C1011301010267800000130101FE3B
:102F2000232E1100EFD00FFE930705002326F1009A
:102F300097D701009387877483A707002324F100A4
:102F40008327C10013850700EFD00FFA8327810084
:102F5000138507008320C10113010102678000006F
:102F600097D701009387477183A707001385070050
:102F700067800000130101FD232611022326A10012
:102F80002324B1002322C100232E01009307A000B7
:102F9000232CF100EFF01FD697D701009387C76D60
:102FA00083A7070003278100636CF714832781013F
:102FB0009387F7FF232CF1008327C10193975700D4
:102FC0000327C100B306F700032781019307070019
:102FD00093972700B387E7009397270017D701003F
:102FE00013070756B387E700130610009385070001
:102FF00013850600EF108004130705008327C10125
:10300000B387E700232EF10083278101E39007FABD
:103010008327C101939757000327C1003307F700A7
:1030200097D701009387C76083A707001306200086
:103030009385070013050700EF10400013070500F4
:103040008327C101B387E700232EF1008327C10145
:10305000939757000327C1003307F70097D7010064
:103060009387475D83A70700130620009385070019
:1030700013050700EF00907C130705008327C101AB
:10308000B387E700232EF1008327C10193975700F0
:103090000327C100B307F7001306400097D50100CE
:1030A0009385C55A13850700EF0050791307050073
:1030B0008327C101B387E700232EF1008327C101D5
:1030C000939757000327C100B307F700130630009A
:1030D00097D501009385055913850700EF001076F9
:1030E000130705008327C101B387E700232EF100F2
:1030F00083274100638607008327410023A0070040
:10310000EFF09FC18327C101138507008320C1020F
:103110001301010367800000130101FD2326110242
:10312000232E010097D701009387475783A70700F5
:10313000639C072297D701009387475483A7070012
:103140001387170097D701009387475323A0E70001
:1031500097D701009387875283A70700232CF1009C
:1031600083278101639C070697D701009387474C0B
:1031700083A7070083A707006386070073700430E6
:103180006F00000097D701009387874A83A7070045
:10319000232AF10097D701009387C74903A70700A7
:1031A00097D701009387C74823A0E70097D701006E
:1031B000938747480327410123A0E70097D70100E1
:1031C0009387074D83A707001387170097D7010040
:1031D0009387074C23A0E700EF10001097D701005A
:1031E0009387874B83A7070003278101636CF7123E
:1031F00097D701009387C74383A7070083A70700DA
:1032000063960700930710006F008000930700008B
:10321000638C070097D70100938707481307F0FFD7
:1032200023A0E7006F00001097D701009387474065
:1032300083A7070083A7C70083A7C7002328F1003F
:103240008327010183A747002326F100032781017B
:103250008327C100637CF70097D701009387C7439A
:103260000327C10023A0E7006F00C00B83270101E3
:103270009387470013850700EFD08FF18327010163
:1032800083A78702638A0700832701019387870149
:1032900013850700EFD0CFEF8327010103A7C702F3
:1032A00097D701009387C73D83A7070063FCE7001A
:1032B0008327010103A7C70297D701009387473CE3
:1032C00023A0E7008327010103A7C7029307070094
:1032D00093972700B387E7009397270017D701003C
:1032E000130707263387E7008327010193874700E9
:1032F0009385070013050700EFD04FD58327010101
:1033000003A7C70297D701009387C71983A70700B0
:1033100083A7C702E36EF7EC93071000232EF1009A
:103320006FF01FED97D701009387C71783A707009A
:1033300003A7C70297D6010093868620930707004C
:1033400093972700B387E70093972700B387F6008A
:1033500003A707009307100063F6E7029307100026
:10336000232EF1006F00000297D701009387C73129
:1033700083A707001387170097D701009387C730EB
:1033800023A0E70097D701009387473083A7070062
:103390006386070093071000232EF1008327C101E5
:1033A000138507008320C102130101036780000019
:1033B000130101FE232E110097D701009387072EDA
:1033C00083A70700638C070097D701009387072C1A
:1033D0001307100023A0E7006F00C01897D7010063
:1033E0009387C72A23A0070097D701009387870BED
:1033F00083A7070083A707032326F100B7A7A5A586
:103400009387575A2324F1008327C10083A707001D
:10341000032781006310F7048327C10093874700C7
:1034200083A70700032781006316F7028327C100E3
:103430009387870083A7070003278100631CF70099
:103440008327C1009387C70083A707000327810054
:103450006302F70697D701009387C70403A7070005
:1034600097D701009387070483A707009387470333
:103470009385070013050700EF4000196F008003D4
:1034800097D701009387C71F83A70700639607009C
:10349000737004306F00000097D701009387471EB8
:1034A00083A707001387F7FF97D701009387471D6E
:1034B00023A0E70097D701009387871C03A7070085
:1034C00097D601009386C6079307070093972700B6
:1034D000B387E70093972700B387F60083A7070019
:1034E000E38007FA97D701009387871903A707009E
:1034F0009307070093972700B387E7009397270068
:1035000017D701001307C703B387E7002322F10091
:103510008327410083A7470003A747008327410073
:1035200023A2E7008327410003A747008327410028
:1035300093878700631CF7008327410083A7470018
:1035400003A747008327410023A2E7008327410008
:1035500083A7470003A7C70097D70100938787F485
:1035600023A0E700130000008320C1011301010222
:1035700067800000130101FD232611022326A1000C
:103580002324B1008327C1006396070073700430C1
:103590006F00000097D701009387C7F083A707004B
:1035A00093878701938507000325C100EFD0CFB132
:1035B00097D70100938707EF83A7070093874700FA
:1035C00013850700EFD0CFBC032781009307F0FFDE
:1035D0006314F70297D701009387C7EC83A707000E
:1035E000938747009385070017D5010013058507CA
:1035F000EFD0CFA56F00400297D70100938707084F
:1036000083A7070003278100B307F700232EF100EB
:103610000325C101EF00900B130000008320C102BD
:103620001301010367800000130101FD232611022D
:103630002326A1002324B1002322C1008327C10037
:1036400063960700737004306F00000097D7010085
:103650009387C70483A7070063960700737004303D
:103660006F00000097D701009387C7E383A7070087
:10367000832681003707008033E7E60023ACE700AC
:1036800097D70100938707E283A7070093878701F5
:10369000938507000325C100EFD04F9B97D701000A
:1036A000938747E083A707009387470013850700A8
:1036B000EFD00FAE032741009307F0FF6314F7022A
:1036C00097D70100938707DE83A7070093874700FA
:1036D0009385070017D501001305C5F8EFD00F97A4
:1036E0006F00400297D70100938747F983A707002F
:1036F00003274100B307F700232EF1000325C10182
:10370000EF00C07C130000008320C10213010103FD
:1037100067800000130101FD232611022326A1006A
:103720002324B1002322C1008327C1006396070030
:10373000737004306F00000097D70100938787D61D
:1037400083A7070093878701938507000325C1009E
:10375000EFD0CF8F97D701009387C7D483A70700F7
:103760009387470013850700EFD08FA203274100FE
:10377000930710006314F70297D70100938787D24D
:1037800083A70700938747009385070017D501009B
:10379000130545EDEFD08F8B6F00400297D70100E6
:1037A0009387C7ED83A7070003278100B307F700BE
:1037B000232EF1000325C101EF004071130000002A
:1037C0008320C1021301010367800000130101FD82
:1037D000232611022326A1008327C10083A7C70047
:1037E00083A7C700232CF10083278101639607007C
:1037F000737004306F000000832781019387870175
:1038000013850700EFD0CF9897D70100938707E97A
:1038100083A70700639E07068327810193874700DC
:1038200013850700EFD0CF968327810103A7C70236
:1038300097D701009387C7E483A7070063FCE700DD
:103840008327810103A7C70297D70100938747E326
:1038500023A0E7008327810103A7C702930707007E
:1038600093972700B387E7009397270017D70100A6
:10387000130707CD3387E70083278101938747002C
:103880009385070013050700EFC05FFC6F00C001C0
:1038900083278101938787019385070017D501004E
:1038A000130585D9EFC09FFA8327810103A7C702BB
:1038B00097D70100938707BF83A7070083A7C70295
:1038C00063F0E70293071000232EF10097D7010061
:1038D0009387C7DB1307100023A0E7006F00800069
:1038E000232E01008327C101138507008320C10215
:1038F0001301010367800000130101FD232611025B
:103900002326A1002324B10097D70100938707D96C
:1039100083A7070063960700737004306F000000F0
:1039200003278100B70700803367F7008327C100B2
:1039300023A0E7008327C10083A7C700232CF10041
:103940008327810163960700737004306F000000C5
:103950000325C100EFD0CF838327810193874700E0
:1039600013850700EFD0CF828327810103A7C70209
:1039700097D701009387C7D083A7070063FCE700B0
:103980008327810103A7C70297D70100938747CFF9
:1039900023A0E7008327810103A7C702930707003D
:1039A00093972700B387E7009397270017D7010065
:1039B000130707B93387E7008327810193874700FF
:1039C0009385070013050700EFC05FE88327810197
:1039D00003A7C70297D701009387C7AC83A7070047
:1039E00083A7C70263F0E70293071000232EF100BC
:1039F00097D70100938787C91307100023A0E7001A
:103A00006F008000232E01008327C101138507006A
:103A10008320C1021301010367800000130101FF2D
:103A20002326A1008327C10063960700737004302A
:103A30006F00000097D70100938787C503A7070091
:103A40008327C10023A0E70097D70100938707C30E
:103A500003A707008327C10023A2E700130000008B
:103A60001301010167800000130101FD23261102EB
:103A70002326A1002324B1008327C10063960700F9
:103A8000737004306F000000832781006396070085
:103A9000737004306F000000EF00103C97D70100F6
:103AA0009387C7BD83A70700232CF10083278100DC
:103AB00003A707009307F0FF6316F700232E01000A
:103AC0006F0000098327C10003A7070097D70100F3
:103AD000938707BC83A707006300F7028327C10011
:103AE00083A74700032781016368F700930710004D
:103AF000232EF1006F00C0058327C10083A7470074
:103B0000032781013307F7408327810083A707003C
:103B1000637CF7028327810003A707008327C10086
:103B200083A6470083278101B387F6403307F70058
:103B30008327810023A0E7000325C100EFF01FEEDB
:103B4000232E01006F00C00093071000232EF10008
:103B5000EF0090348327C101138507008320C10241
:103B6000130101036780000097D70100938707B214
:103B70001307100023A0E700130000006780000077
:103B8000130101FE2326A1008327C100638E0700D5
:103B90008327C100232CF1008327810183A7C70459
:103BA000232EF1006F008000232E01008327C10126
:103BB000138507001301010267800000130101FE55
:103BC0002326A1002324B1008327C100638C0700B2
:103BD0008327C100232EF1008327C1010327810021
:103BE00023A6E70413000000130101026780000010
:103BF000130101FE232E11002326A100EF00002156
:103C000097D701009387C79303A707009307100076
:103C1000E3F6E7FEEFC0DF976FF05FFE130101FCF4
:103C2000232E1102232EA100232CB100232AC10030
:103C30002328D100930707002317F1002326010250
:103C40006F004004032781018327C102B307F700F7
:103C500003C707008326C1018327C102B387F6008B
:103C6000238AE702032781018327C102B307F700F4
:103C700083C70700638007028327C1029387170069
:103C80002326F1020327C1029307F000E3FCE7FAC1
:103C90006F008000130000008327C101A381070487
:103CA000032741019307900063F6E7009307900014
:103CB000232AF1008327C1010327410123A6E7023C
:103CC0008327C1010327410123A8E7048327C101FA
:103CD00023AA07048327C1019387470013850700A0
:103CE000EFC01FB58327C1019387870113850700A4
:103CF000EFC01FB48327C1010327C10123A8E70038
:103D00001307A000832741013307F7408327C10130
:103D100023ACE7008327C1010327C10123A2E702E7
:103D20008327C10123A207048327C10123AC070411
:103D30008327C10123AE0704130000008320C103C1
:103D40001301010467800000130101FE232E1100FE
:103D5000232601006F0080030327C100930707009B
:103D600093972700B387E7009397270017C70100B1
:103D70001307077DB387E70013850700EFC0DFA5B2
:103D80008327C100938717002326F1000327C10072
:103D900093079000E3F2E7FC17D501001305C586F1
:103DA000EFC09FA317D5010013054587EFC0DFA221
:103DB00017D5010013054588EFC01FA217D50100D4
:103DC0001305C588EFC05FA117D5010013058589CC
:103DD000EFC09FA097D701009387878517D7010071
:103DE0001307878223A0E70097D701009387878472
:103DF00017D701001307878223A0E70013000000F4
:103E00008320C1011301010267800000130101FE3C
:103E1000232E11006F008009EFE0DFED97D701003E
:103E20009387C78283A7070093B7170093F7F70F0D
:103E30002326F100EFE05FEE8327C10063980706B9
:103E4000EF00900197D701009387478083A7C700B1
:103E500083A7C7002324F1008327810093874700AD
:103E600013850700EFC0DFB297D701009387C780A3
:103E700083A707001387F7FF97C701009387C77FC2
:103E800023A0E70097C701009387877D83A70700DA
:103E90001387F7FF97C701009387877C23A0E7006C
:103EA000EF00807F03258100EF00C03F97C701002E
:103EB0009387077B83A70700E39007F613000000B2
:103EC0008320C1011301010267800000130101FE7C
:103ED000232E11002326A10097C701009387875C3A
:103EE00083A707000327C10023A2E70097C70100AB
:103EF0009387C77883A707000327C1006378F70279
:103F000097C701009387077303A7070097C70100AE
:103F10009387475983A70700938747009385070036
:103F200013050700EFC05F9A6F00000597C70100F7
:103F30009387077003A7070097C7010093878756E9
:103F400083A70700938747009385070013050700A1
:103F5000EFC09F9797C701009387077483A7070057
:103F60000327C100637AF70097C701009387C772E0
:103F70000327C10023A0E700130000008320C10134
:103F80001301010267800000130101FD23261102C5
:103F9000930705002324B1002317F1008327810034
:103FA000639E07008357E10093972700138507005E
:103FB000EF20C02E930705006F008000832781004B
:103FC000232CF10083278101638A07021305000671
:103FD000EF20C02C232EA1008327C101638A070094
:103FE0008327C1010327810123A8E7026F00400155
:103FF00003258101EF20404A6F008000232E01003D
:104000008327C101638207028327C10103A7070336
:104010008357E10093972700138607009305500A02
:1040200013050700EF20006A8327C10113850700ED
:104030008320C1021301010367800000130101FC0A
:10404000232E1102232C81022326A1002324B10058
:104050002322C100232601028327810083A70700B2
:104060006388071C832781002324F10283278102B0
:1040700083A7470003A747008327810223A2E70005
:104080008327810203A74700832781029387870044
:10409000631CF7008327810283A7470003A747001B
:1040A0008327810223A2E7008327810283A7470099
:1040B00083A7C7002322F102832781002320F10276
:1040C0008327010283A7470003A747008327010234
:1040D00023A2E7008327010203A7470083270102E9
:1040E00093878700631CF7008327010283A747009B
:1040F00003A747008327010223A2E70083270102C9
:1041000083A7470083A7C700232EF1008327C1029E
:10411000939757000327C100B307F7000327C10196
:1041200023A0E7008327C102939757000327C1000C
:10413000B307F7000327C1011307470323A2E700D2
:104140008327C102939757000327C100B307F700E5
:104150000327C1010327870423A4E7008327C102A3
:10416000939757000327C100B307F70003274100C7
:1041700023A6E7008327C102939757000327C100B6
:10418000B307F7000327C1010327C70223A8E700ED
:1041900003274100930730006314F7028327C1010E
:1041A00083A78702638E07008327C1029397570076
:1041B0000327C100B307F7001307200023A6E70079
:1041C0008327C102939757000327C100B307F70065
:1041D0000327C1010327070523AAE7008327C1029C
:1041E000939757000327C100B307F70023AC0700DC
:1041F0008327C10183A607038327C1029397570032
:104200000327C1003304F70013850600EF00C00345
:1042100093070500231EF4008327C102938717002C
:104220002326F1020327C10183274102E316F7E8A1
:104230008327C102138507008320C1030324810360
:104240001301010467800000130101FE2326A10071
:10425000232E01006F00C0018327C1009387170040
:104260002326F1008327C10193871700232EF10035
:104270008327C10003C707009307500AE30EF7FC2A
:104280008327C10193D72700232EF1008327C10183
:104290009397070193D707011385070013010102C4
:1042A00067800000130101FE232E11002326A100C8
:1042B0008327C10083A7070313850700EF20C01DD4
:1042C0000325C100EF20401D130000008320C10121
:1042D0001301010267800000130101FF97C701006D
:1042E0009387073583A7070083A707006396070016
:1042F000930710006F00800093070000638C070095
:1043000097C70100938747391307F0FF23A0E70001
:104310006F00000397C701009387873183A70700C9
:1043200083A7C70083A7C7002326F1008327C10006
:1043300003A7470097C701009387073623A0E7002C
:10434000130000001301010167800000130101FF49
:1043500097C701009387071583A707002326F1005D
:104360008327C10013850700130101016780000046
:10437000130101FF97C701009387C73083A7070088
:1043800063980700930710002326F1006F00400296
:1043900097C701009387873083A7070063980700BA
:1043A000930720002326F1006F00800023260100E0
:1043B0008327C100138507001301010167800000F6
:1043C000130101FD232611022326A1008327C1002A
:1043D000232EF1008327C100638A07128327C101BE
:1043E00003A7C70297C701009387C70B83A70700DE
:1043F00083A7C702637CF7108327C10183A78701C6
:1044000063C2070297C701009387C70983A7070004
:1044100083A7C7021307A0003307F7408327C10112
:1044200023ACE7008327C10183A647018327C1018D
:1044300003A7C7029307070093972700B387E700F6
:104440009397270017C701001307870FB387E7006B
:104450006396F600930710006F008000930700003A
:10446000638A07088327C1019387470013850700E4
:10447000EFC00FD297C701009387C70283A7070039
:1044800003A7C7028327C10123A6E7028327C1012F
:1044900003A7C70297C701009387871E83A707005A
:1044A00063FCE7008327C10103A7C70297C7010088
:1044B0009387071D23A0E7008327C10103A7C70235
:1044C0009307070093972700B387E7009397270088
:1044D00017C701001307C7063387E7008327C10109
:1044E000938747009385070013050700EFC00FB6B9
:1044F0006F00C00197C701009387C7FA83A7070021
:1045000003A7C7028327C10123A6E7021300000007
:104510008320C1021301010367800000130101FD24
:10452000232611022326A1008327C100232CF1009A
:10453000232E01008327C1006386071097C701005F
:10454000938747F683A70700032781016306F700D7
:10455000737004306F0000008327810183A7470533
:1045600063960700737004306F0000008327810199
:1045700083A747051387F7FF8327810123AAE70451
:104580008327810103A7C7028327810183A707052A
:10459000630AF70A8327810183A747056394070A03
:1045A000832781019387470013850700EFC04FBE23
:1045B0008327810103A707058327810123A6E7023B
:1045C0008327810183A7C7021307A0003307F740A1
:1045D0008327810123ACE7008327810103A7C7025A
:1045E00097C701009387C70983A7070063FCE7000B
:1045F0008327810103A7C70297C701009387470854
:1046000023A0E7008327810103A7C70293070700C0
:1046100093972700B387E7009397270017C70100F8
:10462000130707F23387E700832781019387470049
:104630009385070013050700EFC04FA193071000F3
:10464000232EF1008327C101138507008320C102B7
:1046500013010103678000007370043097C70100E5
:104660009387470283A707006384070297C7010067
:10467000938747E383A7070003A74704130717009F
:1046800023A2E70497C701009387C7E183A7070028
:10469000130000006780000097C70100938787FE22
:1046A00083A707006384070497C70100938787DF08
:1046B00083A7070083A74704638A070297C70100FF
:1046C000938747DE83A7070003A747041307F7FF75
:1046D00023A2E70497C701009387C7DC83A70700DD
:1046E00083A747046394070073600430130000003D
:1046F00067800000130101FF97C70100938787DAE5
:1047000083A7070083A787012326F10097C701002D
:10471000938747D983A7070003A7C70297C701005C
:10472000938747D883A707009306A0003387E64006
:1047300023ACE7008327C1001385070013010101A3
:104740006780000097C701009387C7D583A707003C
:10475000638E070097C701009387C7D483A707001C
:1047600003A747051307170023AAE70497C701000B
:10477000938747D383A7070013850700678000004E
:10478000130101FD232611022326A1002324B100D9
:10479000EFF09FEC97C701009387C7D083A707006E
:1047A00083A787056396070897C70100938787CF7C
:1047B00083A707001307100023AEE70483278100B7
:1047C0006388070697C701009387C7CD83A70700B3
:1047D0009387470013850700EFC08F9B0327810055
:1047E0009307F0FF6314F70297C70100938787CB05
:1047F00083A70700938747009385070017C501002B
:10480000130545E6EFC08F846F00400297C7010093
:104810009387C7E683A7070003278100B307F70044
:10482000232EF1000325C101EFF04FEAEFB05FD670
:10483000EFF09FE6EFF05FE297C70100938787C62E
:1048400083A7070083A78705232CF1008327810115
:10485000638C07028327C100638C070097C70100A0
:10486000938747C483A7070023AC07046F00C001E8
:1048700097C70100938707C383A7070003A787058E
:104880001307F7FF23ACE70497C70100938787C19D
:1048900083A7070023AE0704EFF01FE08327810101
:1048A000138507008320C102130101036780000004
:1048B000130101FD232611022326A1002324B100A8
:1048C0002322C1002320D100EFF01FD997C7010098
:1048D000938747BD83A7070003A7C7059307200059
:1048E0006306F70A97C701009387C7BB83A7070032
:1048F00083A687050327C1001347F7FF33F7E600B8
:1049000023ACE70497C701009387C7B983A70700C3
:104910001307100023AEE70483270100638807060E
:1049200097C70100938707B883A7070093874700BD
:1049300013850700EFC0CF85032701009307F0FF21
:104940006314F70297C701009387C7B583A70700D1
:10495000938747009385070017C50100130585D08D
:10496000EFB0DFEE6F00400297C70100938707D1D9
:1049700083A7070003270100B307F700232CF100EA
:1049800003258101EFF08FD4EFB09FC0EFF0DFD0AF
:10499000EFF09FCC83274100638E070097C701008B
:1049A000938747B083A7070003A7870583274100A4
:1049B00023A0E70097C701009387C7AE83A707002E
:1049C00003A7C705930710006316F700232E010005
:1049D0006F00C00297C701009387C7AC83A7070089
:1049E00083A68705032781001347F7FF33F7E60007
:1049F00023ACE70493071000232EF10097C70100B2
:104A0000938747AA83A7070023AE0704EFF0DFC808
:104A10008327C101138507008320C102130101030D
:104A200067800000130101FD232611022326A10047
:104A30002324B1002322C1002320D10093071000BA
:104A4000232EF1008327C1006396070073700430A2
:104A50006F0000008327C100232CF100EFF0DFBFBF
:104A600083270100638A07008327810103A7870545
:104A70008327010023A0E7008327810183A7C705BF
:104A8000232AF100832781011307200023AEE704C6
:104A9000032741009307400063ECE70883274100A8
:104AA0001397270097B7010093874756B307F7007E
:104AB00003A7070097B7010093874755B307F7008F
:104AC000678007008327810103A78705832781006B
:104AD0003367F7008327810123ACE7046F004005AB
:104AE0008327810183A78705138717008327810107
:104AF00023ACE7046F00C0038327810103278100F3
:104B000023ACE7046F00C002032741019307200094
:104B1000630AF700832781010327810023ACE704A0
:104B20006F000001232E01006F00800013000000C1
:104B300003274101930710006316F70A83278101B9
:104B40009387470013850700EFB09FE48327810117
:104B500003A7C70297C70100938787B283A70700FF
:104B600063FCE7008327810103A7C70297C7010001
:104B7000938707B123A0E7008327810103A7C7021A
:104B80009307070093972700B387E70093972700C1
:104B900017C701001307C79A3387E70083278101EE
:104BA000938747009385070013050700EFB01FCADE
:104BB0008327810183A7870263860700737004300F
:104BC0006F0000008327810103A7C70297C7010078
:104BD0009387478D83A7070083A7C70263F4E70085
:104BE000EFB01F9BEFF05FAB8327C1011385070078
:104BF0008320C1021301010367800000130101FC3F
:104C0000232E1102232EA100232CB100232AC10040
:104C10002328D1002326E100930710002326F10268
:104C20008327C10163960700737004306F00000092
:104C30008327C1012324F102EFB0DFAC9307050005
:104C40002322F10283270101638A0700832781025F
:104C500003A787058327010123A0E700832781029B
:104C600083A7C7052320F1028327810213072000B1
:104C700023AEE704032741019307400063ECE708F4
:104C8000832741011397270097B70100938747397E
:104C9000B307F70003A7070097B7010093874738CA
:104CA000B307F700678007008327810203A7870502
:104CB000832781013367F7008327810223ACE70450
:104CC0006F0040058327810283A78705138717009C
:104CD0008327810223ACE7046F00C003832781028E
:104CE0000327810123ACE7046F00C0020327010200
:104CF00093072000630AF7008327810203278101BD
:104D000023ACE7046F000001232601026F0080003E
:104D10001300000003270102930710006314F70E2D
:104D20008327810283A7870263860700737004309C
:104D30006F00000097C701009387479683A707007D
:104D4000639E070683278102938747001385070028
:104D5000EFB01FC48327810203A7C70297C70100D2
:104D60009387079283A7070063FCE70083278102EC
:104D700003A7C70297C701009387879023A0E70086
:104D80008327810203A7C702930707009397270091
:104D9000B387E7009397270017B701001307477AF7
:104DA0003387E700832781029387470093850700B5
:104DB00013050700EFB09FA96F00C0018327810290
:104DC000938787019385070017C501001305C586E2
:104DD000EFB0DFA78327810203A7C70297B70100BF
:104DE0009387476C83A7070083A7C70263FCE7008C
:104DF0008327C100638807008327C10013071000C1
:104E000023A0E7008327410213850700EFB0DF8D61
:104E10008327C102138507008320C1031301010406
:104E200067800000130101FD232611022326A10043
:104E30002324B1008327C1006396070073700430F8
:104E40006F0000008327C100232EF100EFB09F8B7D
:104E500093070500232CF1008327C10183A7C70511
:104E6000232AF1008327C1011307200023AEE704A2
:104E70008327C10183A78705138717008327C101F3
:104E800023ACE70403274101930710006314F70ED6
:104E90008327C10183A787026386070073700430EC
:104EA0006F00000097B701009387477F83A7070033
:104EB000639E07068327C101938747001385070078
:104EC000EFB01FAD8327C10103A7C70297B7010049
:104ED0009387077B83A7070063FCE7008327C10153
:104EE00003A7C70297B701009387877923A0E7003C
:104EF0008327C10103A7C7029307070093972700E1
:104F0000B387E7009397270017B70100130747639C
:104F10003387E7008327C101938747009385070004
:104F200013050700EFB09F926F00C0018327C101F6
:104F3000938787019385070017B501001305C56F97
:104F4000EFB0DF908327C10103A7C70297B7010025
:104F50009387475583A7070083A7C70263FCE70031
:104F600083278100638807008327810013071000CF
:104F700023A0E7008327810113850700EFB0CFF658
:104F8000130000008320C1021301010367800000A9
:104F9000130101FD232611022326A1008327C1004E
:104FA000232CF10083278101639A070097B7010042
:104FB0009387474F83A707006F00800083278101F5
:104FC000232CF100EFF04FE98327810103A7C705E8
:104FD00093072000631CF7008327810123AE070499
:104FE00093071000232EF1006F008000232E010094
:104FF000EFF08FEA8327C101138507008320C102E8
:105000001301010367800000130101FE232E11002C
:1050100023260100EF00500B97B701009387476BE1
:1050200083A70700638A07029308000013080000A3
:1050300093070000130720009306000013060040AA
:1050400097B50100938505FF170500001305852E10
:10505000EFC01FEF2326A1008327C100639607003E
:10506000737004306F0000008327C10013850700B0
:105070008320C1011301010267800000130101FCBC
:10508000232E1102232EA100232CB100232AC100BC
:105090002328D1002326E10083278101639607009E
:1050A000232601026F0080061305C002EF10001FC7
:1050B0002326A1028327C102638A0704EF00D000E0
:1050C0008327C1020327C10123A0E7008327C10270
:1050D0000327810123ACE7008327C1020327410195
:1050E00023AEE7008327C1020327010123A0E702C3
:1050F0008327C1020327C10023A2E7028327C1023D
:105100009387470013850700EFB08FF28327810153
:1051100063960700737004306F0000008327C1029C
:10512000138507008320C103130101046780000079
:10513000130101FC232E1102232EA100232CB10008
:10514000232AC1002328D1002326E10023260102BF
:105150008327C10163960700737004306F0000005D
:1051600097B701009387C75683A70700638C070A88
:10517000832781012320F102832741012322F102A9
:105180008327C1012324F1020327810193075000E3
:1051900063C6E706EFF0CF9D1307050093072000D5
:1051A0006318F70297B701009387875283A7070018
:1051B00013070102930600000326C10093050700B0
:1051C00013850700EFB01FD22326A1026F008005D0
:1051D00097B701009387C74F83A707001307010202
:1051E00093060000130600009305070013850700CF
:1051F000EFB05FCF2326A1026F00C00297B7010076
:105200009387074D83A70700130701029306000049
:10521000032601019305070013850700EFB09FF0F7
:105220002326A1028327C102138507008320C1031F
:105230001301010467800000130101FE2326A10071
:105240008327C100232EF1008327C1006396070046
:10525000737004306F0000008327C10183A707002B
:10526000138507001301010267800000130101FD8F
:10527000232611022326A1002324B10097B70100A1
:105280009387874483A7070083A7C70083A7C70026
:10529000232EF1008327C101938747001385070060
:1052A000EFB00FEF8327C10103A7C70193071000D9
:1052B0006310F7068327C10103A787018327C10075
:1052C000B307F7008326C1000326810093850700FA
:1052D0000325C101EF00802213070500930710008A
:1052E0006318F70213070000930600000326C100AD
:1052F000930500000325C101EFF09FE3232CA100DB
:105300008327810163960700737004306F000000EB
:105310008327C10183A747020325C101E780070056
:10532000130000008320C102130101036780000005
:10533000130101FD232611022326A10093078101F9
:1053400013850700EF00800E232EA1008327810123
:10535000938507000325C101EF00C000EF0000287E
:105360006FF0DFFD130101FD232611022326A100AA
:105370002324B100EFD01F98930781011385070004
:10538000EF004011232EA1008327810163960708B7
:1053900083278100639207020327C1008327C1018D
:1053A00063ECE700EFD05F978325C1010325C100BF
:1053B000EFF0DFEB6F008006832781006380070238
:1053C00097B701009387873083A7070083A707005B
:1053D00093B7170093F7F70F2324F10097B7010055
:1053E0009387072F83A607000327C1008327C101E6
:1053F000B307F74003268100938507001385060055
:10540000EFC01FABEFD05F919307050063980700D3
:10541000EFB00F986F008000EFD01F9013000000D6
:105420008320C1021301010367800000130101FE04
:105430002326A10097B701009387072983A70700B8
:1054400083A7070093B7170093F7F70F1387070099
:105450008327C10023A0E7008327C10083A707009B
:105460006390070297B701009387072683A7070079
:1054700083A7C70083A70700232EF1006F008000D9
:10548000232E01008327C1011385070013010102A8
:1054900067800000130101FD232611022326A100CD
:1054A000EFD09FA4232EA10097B7010093878722F6
:1054B00083A707000327C101637CF700EF00C02B1F
:1054C0008327C1001307100023A0E7006F00C0006E
:1054D0008327C10023A0070097B701009387871F88
:1054E0000327C10123A0E7008327C101138507001B
:1054F0008320C1021301010367800000130101FD35
:10550000232611022326A1002324B1002322C10057
:105510002320D100232E01008327C100032781000F
:1055200023A2E7008327C1000327C10023A8E700C7
:10553000032781008327410063E6E7040327410036
:10554000832701003307F7408327C10083A7870122
:105550006368F70093071000232EF1006F00C00668
:1055600097B701009387871603A707008327C10019
:10557000938747009385070013050700EFB0CFB46A
:105580006F0080040327410083270100637EF7003A
:1055900003278100832701006368F7009307100049
:1055A000232EF1006F00400297B701009387C711C7
:1055B00003A707008327C10093874700938507004F
:1055C00013050700EFB04FB08327C1011385070013
:1055D0008320C1021301010367800000130101FD54
:1055E000232611026F0080158327810063C60714EC
:1055F00083270101232EF1008327C10183A74701DF
:10560000638A07008327C10193874700138507003A
:10561000EFB00FB89307410013850700EFF09FE745
:10562000232CA10083278100130790006368F710E3
:105630001397270097B70100938747A0B307F70098
:1056400003A7070097B701009387479FB307F700A9
:10565000678007000327C1008327C10183A7870153
:10566000B307F7000327C100930607000326810153
:10567000938507000325C101EFF05FE813070500DC
:1056800093071000631CF70A8327C10183A7470211
:105690000325C101E78007008327C10103A7C701D4
:1056A00093071000631CF7080327C1008327C1017B
:1056B00083A78701B307F7001307000093060000D4
:1056C00013860700930500000325C101EFF05FA6D4
:1056D000232AA100832741016392070673700430D7
:1056E0006F0000000327C1008327C10123ACE7003E
:1056F0008327C10183A78701639607007370043075
:105700006F0000008327C10103A787018327810160
:10571000B307F700832681010326810193850700E3
:105720000325C101EFF09FDD6F0040010325C1019A
:10573000EF0090566F0080001300000097B7010043
:10574000938707F983A707001307810093060000DA
:10575000130600009305070013850700EFB05FC52F
:1057600093070500E39207E8130000008320C102BD
:105770001301010367800000130101FD23261102BC
:105780006F00C00E97B70100938707F483A7070047
:1057900083A7C70083A70700232CF10097B7010058
:1057A000938787F283A7070083A7C70083A7C70053
:1057B000232AF100832741019387470013850700BF
:1057C000EFB00F9D8327410183A7470203254101C5
:1057D000E78007008327410103A7C7019307100053
:1057E0006316F7088327410183A7870103278101F7
:1057F000B307F7002328F100032701018327810164
:1058000063F0E704832741010327010123A2E70096
:10581000832741010327410123A8E70097B701002F
:10582000938787EA03A707008327410193874700EF
:105830009385070013050700EFB00F896F00000381
:105840001307000093060000032681019305000062
:1058500003254101EFF0DF8D2326A1008327C1003E
:1058600063960700737004306F00000097B7010063
:10587000938787E583A7070083A70700E39407F0D2
:1058800097B70100938747E483A70700232EF10011
:1058900097B70100938787E303A7070097B7010035
:1058A000938787E223A0E70097B70100938707E279
:1058B0000327C10123A0E700130000008320C102D9
:1058C0001301010367800000130101FF232611006B
:1058D000EFE09FD897B70100938787DF83A7070082
:1058E0006394070A17B50100130585DBEFA0DFEE0F
:1058F00017B50100130505DCEFA01FEE97B70100F7
:10590000938787DC17B70100130787D923A0E70027
:1059100097B70100938787DB17B70100130787D973
:1059200023A0E700130600009305C0001305400004
:10593000EFB0CFA21307050097B70100938747D9AF
:1059400023A0E70097B70100938787D883A70700B4
:1059500063960700737004306F00000097B7010072
:10596000938707D783A707006380070297B70100D3
:10597000938707D683A7070097A501009385856EB7
:1059800013850700EFC0CFC2EFE01FD11300000066
:105990008320C1001301010167800000130101FD94
:1059A000232611022326A1008327C100232EF10004
:1059B0008327C10063960700737004306F000000F6
:1059C000EFE09FC98327C10183A74701B337F000E8
:1059D00093F7F70F232CF100EFE01FCC8327810111
:1059E000138507008320C1021301010367800000B3
:1059F000130101FD232611022326A1008327C100E4
:105A0000232EF1008327C1006396070073700430D2
:105A10006F000000EFE05FC48327C10183A7070286
:105A2000232CF100EFE05FC7832781011385070076
:105A30008320C1021301010367800000130101FDEF
:105A4000232611022326A1002324B1008327C100AD
:105A5000232EF1008327C100639607007370043082
:105A60006F000000EFE05FBF8327C10103278100C3
:105A700023A0E702EFE05FC2130000008320C10211
:105A80001301010367800000130101FE232E1100A2
:105A90001305C001EF0090002326A1008327C10059
:105AA000638E07008327C10023A007008327C1005E
:105AB0009387470013850700EFA01FD28327C100FB
:105AC000138507008320C1011301010267800000D4
:105AD000130101FC232E11022326A1002324B1006F
:105AE0002322C1002320D1008327C1002324F102F7
:105AF0002322010203274100B70700FFB377F70015
:105B000063860700737004306F0000008327410034
:105B100063960700737004306F000000EFE05F854C
:105B2000930705006396070083270100639607002B
:105B3000930710006F008000930700006396070032
:105B4000737004306F000000EFD0CF9A832781027A
:105B500083A707002320F102832581000325C100CC
:105B6000EF00804103270102832781003367F7009C
:105B700083274100B377F70003274100631CF70236
:105B80000327010283278100B367F7002326F10270
:105B90008327810203A707008327410093C7F7FFEC
:105BA0003377F7008327810223A0E7002320010039
:105BB0006F00400483270100638807028327810266
:105BC0009386470003274100B7070005B367F70036
:105BD000032601009385070013850600EFD0DFA49C
:105BE000232601026F0000018327810283A707009B
:105BF0002326F102EFD04F92232EA100832701002C
:105C0000638407088327C10163940700EFA05F98AE
:105C1000EFE05FAE2326A1020327C102B70700020F
:105C2000B377F70063980704EFE01FA3832781028F
:105C300083A707002326F1020327C102832741001F
:105C4000B377F700032741006310F702832781022F
:105C500003A707008327410093C7F7FF3377F700B7
:105C60008327810223A0E700EFE01FA39307100022
:105C70002322F1020327C102B70700019387F7FF30
:105C8000B377F7002326F1028327C10213850700AB
:105C90008320C1031301010467800000130101FB8D
:105CA00023261104232EA100232CB100232AC10096
:105CB0002328D1002326E1008327C101232AF102F2
:105CC000232C0102232801028327C10163960700C8
:105CD000737004306F00000003278101B70700FFD5
:105CE000B377F70063860700737004306F0000001D
:105CF0008327810163960700737004306F000000F2
:105D0000EFE00FE793070500639607008327C100C4
:105D100063960700930710006F0080009307000050
:105D200063960700737004306F000000EFC09FFCA3
:105D30008327410383A707002326F10203260101DD
:105D4000832581010325C102EF00404B2324A102DA
:105D500083278102638C07028327C102232EF1026D
:105D60002326010083274101638807088327410315
:105D700003A707008327810193C7F7FF3377F70055
:105D80008327410323A0E7006F0000078327C1009A
:105D9000639807008327C102232EF1026F00C0051C
:105DA00083274101638A070003278103B7070001A6
:105DB000B367F700232CF10283270101638A0700F0
:105DC00003278103B7070004B367F700232CF10210
:105DD000832741039386470003278101832781039B
:105DE000B367F7000326C1009385070013850600FB
:105DF000EFD09F83232E0102EFC01FF22322A102C6
:105E00008327C10063880708832741026394070042
:105E1000EFA00FF8EFE01F8E232EA1020327C1038E
:105E2000B7070002B377F700639C0704EFE0DF8257
:105E30008327410383A70700232EF10203260101D4
:105E4000832581010325C103EF00403B9307050033
:105E5000638407028327410163800702832741038C
:105E600003A707008327810193C7F7FF3377F70064
:105E70008327410323A0E700EFE01F8223280102CC
:105E80000327C103B70700019387F7FFB377F70034
:105E9000232EF1028327C103138507008320C10449
:105EA0001301010567800000130101FD2326110283
:105EB0002326A1002324B1008327C100232EF10053
:105EC0008327C10063960700737004306F000000E1
:105ED00003278100B70700FFB377F7006386070049
:105EE000737004306F000000EFE00FF78327C101EB
:105EF00083A70700232CF1008327C10103A7070014
:105F00008327810093C7F7FF3377F7008327C10109
:105F100023A0E700EFE04FF88327810113850700F6
:105F20008320C1021301010367800000130101FDFA
:105F3000232611022326A1008327C100232EF1006E
:105F4000EFA04FFC93070500232CF1008327C1012C
:105F500083A70700232AF100832781011385070007
:105F6000EFA08FF883274101138507008320C1022A
:105F70001301010367800000130101FB23261104B4
:105F80002326A1002324B100232C01028327C10072
:105F90002328F102232A01028327C1006396070008
:105FA000737004306F00000003278100B70700FF03
:105FB000B377F70063860700737004306F0000004A
:105FC00083270103938747002326F1028327C10219
:105FD000938787002324F102EFC0DFD18327C1021A
:105FE00083A7C700232EF1028327010303A707001D
:105FF000832781003367F7008327010323A0E7008D
:106000006F00000E8327C10383A747002322F102FC
:106010008327C10383A707002320F102232A01025B
:1060200003270102B70700FFB377F700232EF10023
:1060300003270102B70700019387F7FFB377F70043
:106040002320F1020327C101B7070004B377F7004B
:10605000639207028327010303A707008327010236
:10606000B377F7006388070293071000232AF10231
:106070006F0040028327010303A707008327010263
:10608000B377F700032701026316F70093071000A8
:10609000232AF10283274103638007040327C101F8
:1060A000B7070001B377F700638A0700032781036E
:1060B00083270102B367F700232CF1028327010332
:1060C00003A70700B7070002B367F700938507002F
:1060D0000325C103EFD05F8283274102232EF10203
:1060E0000327C10383278102E31EF7F083270103FF
:1060F00003A707008327810393C7F7FF3377F700D0
:106100008327010323A0E700EFC01FC183270103FA
:1061100083A70700138507008320C104130101052D
:1061200067800000130101FD232611022326A10030
:106130008327C100232EF1008327C10193874700E5
:10614000232CF100EFC01FBB6F00400383278101A8
:1061500003A7C70083278101938787006316F70091
:10616000737004306F0000008327810183A7C7008C
:10617000B705000213850700EFD00FF883278101D0
:1061800083A70700E39407FC0325C101EF00C0309B
:10619000EFC09FB8130000008320C1021301010368
:1061A00067800000130101FE232E11002326A100A9
:1061B0002324B100832581000325C100EFF0DFDB3C
:1061C000130000008320C101130101026780000059
:1061D000130101FE232E11002326A1002324B10068
:1061E000832581000325C100EFF01FCC13000000C0
:1061F0008320C1011301010267800000130101FE29
:106200002326A1002324B1002322C100232E010054
:1062100083274100639007020327C1008327810081
:10622000B377F7006386070293071000232EF1006F
:106230006F0000020327C10083278100B377F700B6
:10624000032781006316F70093071000232EF10047
:106250008327C10113850700130101026780000035
:10626000130101FE2326A1008327C100232CF10086
:106270008327C10063960700232E01006F000001F1
:106280008327810183A78701232EF1008327C10182
:10629000138507001301010267800000130101FC50
:1062A000232E11022326A10023220102EFC09FA466
:1062B000973703009387474383A70700639C070032
:1062C000EF00002C97370300938707421307100055
:1062D00023A0E7008327C100638A07029307800099
:1062E000138707008327C100B387E7002326F10047
:1062F0008327C10093F73700638A07008327C10013
:1063000093F7C7FF938747002326F1008327C10037
:10631000638207160327C100B79701009387B7FF71
:1063200063EAE714973703009387073B2324F102BE
:10633000973703009387473A83A707002326F10284
:106340006F0080018327C1022324F1028327C10249
:1063500083A707002326F1028327C10283A74700F2
:106360000327C10063F8E7008327C10283A7070062
:10637000E39A07FC0327C102973703009387473648
:10638000630AF70E8327810283A7070013078000A3
:10639000B387E7002322F1028327C10203A7070086
:1063A0008327810223A0E7008327C10203A74700B8
:1063B0008327C100B307F7401307800013171700A6
:1063C0006378F7080327C1028327C100B307F700EA
:1063D000232EF1008327C10203A747008327C100B2
:1063E0003307F7408327C10123A2E7008327C102B7
:1063F0000327C10023A2E7008327C10183A7470029
:10640000232CF100973703009387072D2320F102F7
:106410006F0000018327010283A707002320F102F8
:106420008327010283A7070083A747000327810171
:10643000E3E2E7FE8327010203A707008327C101E8
:1064400023A0E700832701020327C10123A0E7005F
:1064500097A701009387470603A707008327C10278
:1064600083A747003307F74097A701009387C70426
:1064700023A0E700EFC05F8A8327410263940700EF
:10648000EF10801783274102138507008320C10383
:106490001301010467800000130101FD232611028E
:1064A0002326A1008327C100232CF1008327C100EC
:1064B0006382070A93078000B307F0400327810136
:1064C000B307F700232CF10083278101232AF10071
:1064D000EFC05F828327410183A747002328F10093
:1064E000973703009387471F232EF1006F000001A9
:1064F0008327C10183A70700232EF1008327C10151
:1065000083A7070083A7470003270101E3E2E7FE13
:106510008327C10103A707008327410123A0E700C8
:106520008327C1010327410123A0E70083274101FD
:1065300003A7470097A70100938707F883A70700E1
:106540003307F70097A70100938707F723A0E70019
:10655000EFC08FFC130000008320C1021301010370
:106560006780000097A70100938707F583A70700BE
:10657000138507006780000013000000678000009B
:10658000130101FF97A701009387471593F7C7FFF2
:106590002326F10097370300938707140327C100D0
:1065A00023A0E700973703009387071323A2070070
:1065B000973703009387C712379701001307C7FF68
:1065C00023A2E700973703009387871123A00700D2
:1065D0008327C1002324F10083278100379701001E
:1065E0001307C7FF23A2E7008327810017370300A3
:1065F0001307070F23A0E700130000001301010198
:1066000067800000130101FE2326A1002324B100AE
:106610002322C10083278100232EF1008327C1009C
:10662000232CF1000327C10083278100B367F70003
:1066300093F73700639607066F00C0028327C101F6
:1066400003A707008327810123A0E7008327810197
:1066500093874700232CF1008327C10193874700CC
:10666000232EF100832741009387D7FF0327C10022
:10667000B307F70003278101E362F7FC6F004002D4
:106680000327C10193071700232EF10083278101FF
:1066900093861700232CD100034707002380E700CF
:1066A0000327C10083274100B307F70003278101B7
:1066B000E368F7FC8327C10013850700130101027B
:1066C00067800000130101FE2326A1002324B100EE
:1066D0002322C1000327C10083274100B367F700CD
:1066E00093F73700639807068327810093F7F70F26
:1066F000232AF10083274101939787000327410153
:10670000B367F700232AF10083274101939707011C
:1067100003274101B367F700232AF1008327C10053
:10672000232EF1006F0080018327C10113874700EA
:10673000232EE1000327410123A0E7000327C10026
:1067400083274100B307F7000327C101E36EF7FC7D
:106750006F00C0038327C100232CF1006F00C0012C
:106760008327810113871700232CE1000327810071
:106770001377F70F2380E7000327C1008327410029
:10678000B307F70003278101E36CF7FC8327C100FF
:10679000138507001301010267800000130101FE49
:1067A0002326A1008327C100232EF1006F000001E2
:1067B0008327C10193871700232EF1008327C1018E
:1067C00083C70700E39607FE0327C1018327C100A3
:1067D000B307F7401385070013010102678000002B
:1067E000130101FE2326A1002324B1008327C10049
:1067F000138717002326E10083C70700A30FF100CA
:1068000083278100138717002324E10083C7070033
:10681000230FF1008347F101638807000347F1016B
:106820008347E101E304F7FC0347F1018347E101FA
:10683000B307F740138507001301010267800000CA
:10684000130101FE2326A1002324B1008327C100E8
:10685000232EF10013000000032781009307170087
:106860002324F1008327C10193861700232ED10032
:10687000034707002380E70083C70700E39E07FC68
:106880008327C10013850700130101026780000000
:10689000130101FE2326A100232E0100232C010059
:1068A0006F0000018327C100938717002326F100A2
:1068B0008327C10003C7070093070002E304F7FE24
:1068C0008327C10003C707009307D002630AF700BC
:1068D0008327C10003C707009307B0026312F706BE
:1068E0008327C10083C70700938737FD93B717003D
:1068F00093F7F70F232CF1008327C100938717002C
:106900002326F1006F00C0030327C101930707008E
:1069100093972700B387E70093971700232EF10082
:106920008327C100138717002326E10083C70700D0
:10693000938707FD0327C101B307F700232EF1005A
:106940008327C10083C70700E39007FC83278101E9
:10695000638807008327C101B307F0406F00800000
:106960008327C1011385070013010102678000001E
:10697000130101FE2326A10097370300938787D8D0
:1069800083A707009386170017370300130787D7DD
:106990002320D7000327C1001377F70F9736030092
:1069A000938646DAB387F6002380E7000327C10009
:1069B0009307A000630CF70097370300938787D4F1
:1069C00003A7070093070004631EF704973703002B
:1069D000938747D7232EF1006F00C0038327C1019F
:1069E00013871700232EE10003C70700B70710F035
:1069F000938707F023A0E70097370300938787D09A
:106A000083A707001387F7FF97370300938787CF84
:106A100023A0E700973703009387C7CE83A707001B
:106A2000E39E07FA93070000138507001301010294
:106A300067800000130101EB232611142324811425
:106A40002322911423202115232E3113232C4113AB
:106A5000232A5113232EA100232CB1002328C10087
:106A6000232AD1002326E1002324F100232201015F
:106A7000232601128327C100138A0700930A00000E
:106A8000832701010328410113060A0093860A00A7
:106A90001385070093050800EF1050369307050093
:106AA0001388050013860700930608008327C11288
:106AB000138717002326E112130706009397270078
:106AC00093060113B387F60023AEE7EE8327C100D8
:106AD00013840700930400008327410113870400F7
:106AE00063E8E70483274101138704006398E70004
:106AF000832701011307040063ECE7028327C10029
:106B00001389070093090000130609009386090002
:106B10000325010183254101EF10805093070500F3
:106B2000138805002328F100232A01016FF09FF448
:106B3000130000006F0040018327C10183258101FC
:106B400003254100E7800700832781001387F7FFB3
:106B50002324E1000327C112E340F7FE6F00400544
:106B60008327C1129397270013070113B307F70078
:106B700003A7C7EF8327C11293972700930601133A
:106B8000B387F60083A6C7EF9307900063F6D7009C
:106B9000930770056F00800093070003B387E70039
:106BA0000327C1018325810113850700E700070042
:106BB0008327C1121387F7FF2326E112E342F0FA7D
:106BC000130000008320C114032481148324411482
:106BD000032901148329C113032A8113832A411332
:106BE0001301011567800000130101FF2326A10096
:106BF0002324B10083268100130710006356D702B7
:106C00008327C10083A707009387770093F787FF47
:106C1000938687000327C1002320D70003A84700DD
:106C200083A707006F0000050327810063040702A4
:106C30000327C10003270700130647008326C1006E
:106C400023A0C600032707009307070013080000CE
:106C50006F0040020327C100032707001306470007
:106C60008326C10023A0C60003270700930707005F
:106C700013080000138507009305080013010101A4
:106C800067800000130101FF2326A1002324B10027
:106C900083268100130710006356D7028327C100A3
:106CA00083A707009387770093F787FF9386870072
:106CB0000327C1002320D70003A8470083A70700AC
:106CC0006F00800503278100630607020327C100C8
:106CD00003270700130647008326C10023A0C60030
:106CE00003270700930707001357F741130807000E
:106CF0006F0080020327C100032707001306470027
:106D00008326C10023A0C6000327070093070700BE
:106D10001357F74113080700138507009305080070
:106D20001301010167800000130101FC232E1102F1
:106D3000232C8102232A91022326A1002324B100BF
:106D40002322C1002320D1006F0040026300043CD5
:106D500083274100938717002322F1008327C10076
:106D60008325810013050400E78007008327410085
:106D700083C707001384070093075002E318F4FC4D
:106D800083274100938717002322F10083274100C6
:106D90002328F10093070002A30BF1009307F0FFF3
:106DA000232EF1009307F0FF232CF1002320010292
:106DB00083274100138717002322E10083C70700C0
:106DC000138407009307D4FD130750056360F7325F
:106DD00013972700979701009387C729B307F700F8
:106DE00003A70700979701009387C728B307F70009
:106DF000678007009307D002A30BF1006FF05FFBE1
:106E000093070003A30BF1006FF09FFA232C0100FE
:106E1000032781019307070093972700B387E700B3
:106E200093971700B307F400938707FD232CF10015
:106E30008327410083C70700138407009307F002EC
:106E400063D287049307900363CE870283274100B0
:106E5000938717002322F1006FF09FFB8327010027
:106E6000138747002320E10083A70700232CF100AC
:106E70006F0080018327C101E3DC07F2232E0100AC
:106E80006FF01FF3130000008327C101E3D207F264
:106E900083278101232EF1009307F0FF232CF100BB
:106EA0006FF01FF183270102938717002320F1025F
:106EB0006FF01FF083270100138747002320E100B4
:106EC00083A707000327C1008325810013850700DE
:106ED000E70007006F004023832701001387470066
:106EE0002320E10083A40700639604009794010027
:106EF0009384C4178327C1016350F00803477101CD
:106F00009307D002630AF706832781019385070060
:106F100013850400EF10800E130705008327C101BD
:106F2000B387E740232EF1006F00400283477101D1
:106F30000327C1008325810013850700E7000700B0
:106F40008327C1019387F7FF232EF1008327C10117
:106F5000E34EF0FC6F0040028327C10083258100CF
:106F600013050400E7800700938414008327C10100
:106F70009387F7FF232EF10083C7040013840700D3
:106F80006300040483278101E3C807FC8327810190
:106F90009387F7FF232CF10083278101E3DE07FAB3
:106FA0006F0000028327C1008325810013050002C2
:106FB000E78007008327C1019387F7FF232EF100A5
:106FC0008327C101E340F0FE6F0000149307010026
:106FD0008325010213850700EFF0DFCA9307050040
:106FE000138805002324F10223260103832781024D
:106FF0000328C1029307080063D607048327C10052
:10700000832581001305D002E780070083258102D4
:107010000326C1029307000013080000B386B7409F
:107020001385060033B5A7003307C840B307A74050
:107030001387070093870600130807002324F10233
:10704000232601039307A0002322F1026F004006CC
:107050009307A0002322F1026F0000049307800031
:107060002322F1026F004003930710002320F10256
:107070008327C1008325810013050003E7800700F3
:107080008327C1008325810013058007E78007005F
:10709000930700012322F1029307010083250102D7
:1070A00013850700EFF05FB42324A1022326B10269
:1070B0000327410283477101138807008327C10119
:1070C000032681028326C102832581000325C10096
:1070D000EFF05F966F0040038327C1008325810096
:1070E00013050400E78007006F0000028327C1003A
:1070F0008325810013055002E780070083270101E3
:107100002322F100130000006FF05FC6130000009F
:107110008320C10303248103832441031301010459
:1071200067800000130101FF2326A100B70710F0BC
:10713000938707F20327C10023A0E7006F00000038
:10714000130101FB232611022326A100232AB102E9
:10715000232CC102232ED1022320E1042322F10497
:10716000232401052326110593070105938747FE74
:10717000232EF1008327C101938607000326C10057
:107180009305000017F5FFFF1305C57EEFF0DFB98B
:1071900093070000138507008320C1021301010536
:1071A00067800000130101FE2326A1002324B10003
:1071B0002322710083278100232EF1008327C10140
:1071C00083A707000327C1001377F70F2380E70089
:1071D0008327C10183A70700138717008327C101F5
:1071E00023A0E700130000001301010267800000E4
:1071F000130101FA232E11022326A1002324B1003A
:107200002324C1042326D1042328E104232AF104E2
:10721000232C0105232E1105930701062322F102D9
:107220009307410193054101170600001306C6F7B5
:1072300037F7FFFF9346F7FF37150000130505806A
:107240003388A5003378E8001368783B23A0070152
:107250003305A6003377E5001367773323A2E700F1
:1072600033F7D500931547013787030013073739E4
:1072700033E7E50023A4E7003377D60093164701F0
:10728000370703001307770633E7E60023A6E70076
:107290000F1000008327C1002326F1029307010687
:1072A000938787FE2324F10203278102930741017C
:1072B000138507009307C10093060700032681008A
:1072C00093850700EFF05FA68327C10023800700A6
:1072D0008327C100138707008327C102B307F74044
:1072E000138507008320C103130101066780000096
:1072F000130101FF370510F0130545F403250500C0
:107300002326A100370510F0130505F40325050019
:107310002324A100370510F0130545F403250500CB
:107320008328C100E398A8FC0325C10013030500CE
:107330009303000013170300930600000325810048
:107340009305050013060000B3E7B6003368C700D5
:10735000370710F0130587F4B7150000938505FA79
:1073600013060000B386B70093880600B3B8F80090
:107370003307C800B387E800138707009387060028
:10738000130807002320F500232205011300000045
:107390001301010167800000130101FF2326110082
:1073A000EFF01FF59307000873A0473013000000AB
:1073B0008320C1001301010167800000130101FE59
:1073C000232E11002326A10017950100130505E0C7
:1073D000EFF01FD7130000008320C1011301010249
:1073E00067800000130101FE232E11002326A10057
:1073F00017950100130505DEEFF09FD41300000080
:107400008320C1011301010267800000130101FD07
:10741000232611022326A100232E01006F00400124
:10742000130000008327C10193871700232EF1006A
:107430000327C101B717000093877738E3D2E7FE2F
:1074400017950100130585D9EFF09FCF6FF0DFFC92
:10745000130101FF2326110013050000EF00001C9B
:10746000130000008320C1001301010167800000A8
:10747000130101FE232E110023260100EF00D02C62
:107480001307050093071000630EF700179501001E
:10749000130545D5EFF0DFCA8327C10093E7270026
:1074A0002326F1008327C100138507008320C10133
:1074B0001301010267800000130101FE232E110059
:1074C00023260100EFF0DFF81707000013078706F7
:1074D000930600001306100093054006179501005F
:1074E000130505D2EFD09FB92326A1008327C10041
:1074F00063820702EFB05F9F930705001307000048
:107500009306000013860700930510000325C100B1
:10751000EFD01FC223240100EFB00FF0930700004B
:10752000138507008320C101130101026780000059
:10753000130101FD232611022326A10097970100C4
:10754000938787F683A7070013874706979701005D
:10755000938787F523A0E70097970100938707F5A6
:1075600083A707001387470697970100938707F4BF
:1075700023A0E70097970100938707F303A707006D
:107580009307F07C63DEE704979701009387C7F1C8
:1075900083A7070013870783979701009387C7F096
:1075A00023A0E700EFF0DFEC232EA1008327C10129
:1075B000639E070097970100938747EF03A7070093
:1075C000B71700009387F77663D0E7028327C101DE
:1075D00013850700EFF01FB5EFB00FEF6F0000014C
:1075E000130000006F008000130000008320C10220
:1075F0001301010367800000737004306F00000006
:107600001300000067800000130101FF2326A10082
:107610002324B100737004306F000000130101FED9
:10762000232E11002326A100930800001308000058
:10763000930700000327C100972603009386861452
:107640001306004097950100938545BC170500007F
:107650001305C516EFA0DF8E930800001308000085
:10766000930700000327C100972603009386A61105
:1076700013060040979501009385C5B917050000D2
:107680001305C531EFA0DF8B93080000130800003D
:10769000930700000327C100972603009386C60EB8
:1076A0001306004097950100938545B71705000024
:1076B0001305C54CEFA0DF889308000013080000F5
:1076C000930700000327C100972603009386E60B6B
:1076D00013060040979501009385C5B41705000077
:1076E00013054568EFA0DF8593080000130800002C
:1076F000930700000327C10097260300938606091D
:107700001306004097950100938545B217050000C8
:107710001305C50AEFA0DF829308000013080000DC
:10772000930700000327C1009726030093862606CF
:1077300013060040979501009385C5AF170500001B
:107740001305C525EFA0CFFF930800001308000024
:10775000930700000327C100972603009386460382
:107760001306004097950100938545AD170500006D
:107770001305C540EFA0CFFC9308000013080000DC
:10778000930700000327C100972603009386660035
:1077900013060040979501009385C5AA17050000C0
:1077A0001305455CEFA0CFF9130000008320C10151
:1077B0001301010267800000130101FC232E110256
:1077C000232C81022326A100231701029797010091
:1077D0009387C7A783A707002322F1029797010089
:1077E000938707A783A707002320F102979701003B
:1077F000938747A683A70700232EF1008327410222
:10780000032701029305070013850700EF10002FDF
:1078100093070500138707008327C101938507009D
:1078200013050700EF10D04593070500232AF10048
:107830008327C1002324F10297970100938707A1B2
:1078400083A707002322F10297970100938747A09F
:1078500083A707002320F102979701009387879F52
:1078600083A70700232EF10083274102032701028B
:107870009305070013850700EF10402893070500C4
:10788000138707008327C1019385070013050700AD
:10789000EF10103F93070500232CF100832781018F
:1078A000032741019305070013850700EF1050746B
:1078B000930705009305000013850700EF10902F34
:1078C0009307050063DA070403278101B7070080E7
:1078D000B347F7000327410193050700138507000D
:1078E000EF101071930705001387070013041000B1
:1078F000979701009387479683A507001305070014
:10790000EF10901E930705006344F000130400007D
:107910009377F40F6F0080048327810103274101CF
:107920009305070013850700EF10906C930705007F
:107930001387070013041000979701009387C791DE
:1079400083A5070013050700EF10101A9307050021
:107950006344F000130400009377F40F638607007C
:10796000930710002317F1028317E102E39607EC57
:107970008327810283D707009397070193D70701D5
:107980009387170013970701135707018327810275
:107990002390E7006FF05FEA130101FC232E110230
:1079A000232C81022326A1002317010297970100AF
:1079B0009387C78A83A707002322F10297970100C4
:1079C0009387078A83A707002320F1029797010076
:1079D0009387478983A70700232EF100832741025D
:1079E000032701029305070013850700EF10405697
:1079F00093070500138707008327C10193850700BC
:107A000013050700EF10D02793070500232AF10084
:107A10008327C1002324F1029797010093870784ED
:107A200083A707002322F1029797010093874783DA
:107A300083A707002320F10297970100938787828D
:107A400083A70700232EF1008327410203270102A9
:107A50009305070013850700EF10804F930705007B
:107A6000138707008327C1019385070013050700CB
:107A7000EF10102193070500232CF10083278101CB
:107A8000032741019305070013850700EF105056A7
:107A9000930705009305000013850700EF10901170
:107AA0009307050063DA070403278101B707008005
:107AB000B347F7000327410193050700138507002B
:107AC000EF101053930705001387070013041000ED
:107AD000978701009387477883A507001305070060
:107AE000EF109000930705006344F00013040000BA
:107AF0009377F40F6F0080048327810103274101EE
:107B00009305070013850700EF10904E93070500BB
:107B10001387070013041000978701009387C7732A
:107B200083A5070013050700EF10007C93070500ED
:107B30006344F000130400009377F40F638607009A
:107B4000930710002317F1028317E102E39607EC75
:107B50008327810283D707009397070193D70701F3
:107B60009387170013970701135707018327810293
:107B70002390E7006FF05FEA130101FB2326110455
:107B8000232481042326A1009307A000232AF102C5
:107B9000231D01028327C1002328F102832741030B
:107BA0009397270013850700EFE04FEF2326A102EC
:107BB000930700002324F1022322F102232EF10077
:107BC000232E01026F0080078326C1018327C10392
:107BD000939727000327C1023304F700978701001A
:107BE0009387876883A5070013850600EF0010714F
:107BF000930705002320F4000327C10197870100A4
:107C00009387876683A5070013050700EF00106FB1
:107C100093070500138707008327810293850700D8
:107C200013050700EF00906D930705002324F10270
:107C30008327C10393871700232EF1020327C10373
:107C400083274103E362F7F8232E01026F00C0038C
:107C50008327C103939727000327C102B307F700C7
:107C600083A7070003274102930507001385070038
:107C7000EF00D068930705002322F1028327C10398
:107C800093871700232EF1020327C10383274103A3
:107C9000E360F7FC83278102032741029305070075
:107CA00013850700EF10D034930705002320F1025D
:107CB000832701029305000013850700EF10806FF2
:107CC0009307050063DA070203270102130410007B
:107CD000978701009387875983A50700130507003D
:107CE000EF10406D9307050063C407001304000004
:107CF0009377F40F6F0000030327010213041000B1
:107D0000978701009387475583A507001305070050
:107D1000EF10805D930705006344F000130400003A
:107D20009377F40F6386070093071000231DF10279
:107D30008317A103E39E07E68327010383D7070088
:107D40009397070193D707019387170013970701AC
:107D500013570701832701032390E7006FF05FE5C6
:107D6000130101FB23261104232481042326A100EF
:107D70009307A000232AF102231D01028327C100DB
:107D80002328F102832741039397270013850700D7
:107D9000EFE0CFD02326A102930700002324F102B5
:107DA0002322F102232EF100232E01026F0080070F
:107DB0008326C1018327C103939727000327C102AC
:107DC0003304F700978701009387874A83A507004C
:107DD00013850600EF10C06A930705002320F40006
:107DE0000327C101978701009387874883A5070070
:107DF00013050700EF10C0689307050013870700FD
:107E0000832781029385070013050700EF00104FB9
:107E1000930705002324F1028327C10393871700EA
:107E2000232EF1020327C10383274103E362F7F8FE
:107E3000232E01026F00C0038327C10393972700FD
:107E40000327C102B307F70083A7070003274102F6
:107E50009305070013850700EF00504A93070500BC
:107E60002322F1028327C10393871700232EF102F7
:107E70000327C10383274103E360F7FC83278102C3
:107E8000032741029305070013850700EF105016E2
:107E9000930705002320F1028327010293050000C8
:107EA00013850700EF1000519307050063DA0702FE
:107EB0000327010213041000978701009387073BF3
:107EC00083A5070013050700EF10C04E93070500B8
:107ED00063C40700130400009377F40F6F000003DE
:107EE0000327010213041000978701009387C73608
:107EF00083A5070013050700EF10003F9307050057
:107F00006344F000130400009377F40F63860700C6
:107F100093071000231DF1028317A103E39E07E6D8
:107F20008327010383D707009397070193D707019E
:107F3000938717001397070113570701832701033E
:107F40002390E7006FF05FE5130101FF9307100036
:107F50002326F100232401006F0080081727030067
:107F6000130747828327810093971700B307F70011
:107F700083D70700139707011357070197260300BC
:107F8000938646818327810093971700B387F60075
:107F900083D707006314F700232601001717030097
:107FA0001307477E8327810093971700B307F700D5
:107FB00083D707001397070113570701971603008C
:107FC0009386467D8327810093971700B387F60039
:107FD0002390E70083278100938717002324F10073
:107FE0000327810093077000E3DAE7F68327C100D7
:107FF000138507001301010167800000B305B50078
:10800000930705006386B70003C7070063160700E0
:108010003385A74067800000938717006FF09FFEAD
:10802000130101FD23229102232A5101232611026B
:108030002324810223202103232E3101232C4101FB
:108040002328610123267101232481012322910128
:108050002320A101930A050093840500639E06383E
:108060001304060093090500178901001309092864
:1080700063F8C512B7070100138B05006378F6108B
:108080001307F00F3337C70013173700B357E60055
:108090003309F900834609003387E600930600029E
:1080A000B386E640638C0600B394D40033D7EA006D
:1080B0003314D600336B9700B399DA00935A040156
:1080C00093850A0013050B00EF10504113090500BA
:1080D00093850A00931B040113050B00EF10903BDE
:1080E00093DB0B01930405009305050013850B003A
:1080F000EF1090371319090193D70901B367F900FD
:10810000138A040063FEA700B3878700138AF4FF75
:1081100063E8870063F6A700138AE4FFB38787004C
:10812000B384A74093850A0013850400EF10103B29
:108130001309050093850A0013850400EF1090359C
:10814000939909019304050093050500131909018A
:1081500013850B0093D90901EF101031B369390170
:108160001386040063FCA900B30934011386F4FFED
:1081700063E6890063F4A9001386E4FF13140A017F
:108180003364C400130A00006F000013B707000136
:1081900013070001E36CF6EE130780016FF01FEF89
:1081A000138A0600631A06009305000013051000E9
:1081B000EF10502E13040500B7070100637EF41280
:1081C0009307F00F63F48700130A8000B35744014C
:1081D0003309F900034709009306000233074701FA
:1081E000B386E64063940612B3848440130A1000F9
:1081F000135B040193050B0013850400EF10102E90
:108200001309050093050B0013850400931B04015B
:10821000EF10502893DB0B01930405009305050034
:1082200013850B00EF1050241319090193D709018E
:10823000B367F900938A040063FEA700B387870041
:10824000938AF4FF63E8870063F6A700938AE4FF4C
:10825000B3878700B384A74093050B001385040000
:10826000EF10D0271309050093050B0013850400B8
:10827000EF1050229399090193040500930505001E
:108280001319090113850B0093D90901EF10D01DB3
:10829000B36939011386040063FCA900B3093401F2
:1082A0001386F4FF63E6890063F4A9001386E4FFF4
:1082B00013940A013364C4001305040093050A00F3
:1082C0008320C10203248102832441020329010285
:1082D0008329C101032A8101832A4101032B010162
:1082E000832BC100032C8100832C4100032D01004E
:1082F0001301010367800000B7070001130A0001A2
:10830000E366F4EC130A80016FF05FEC3314D400E1
:1083100033DAE400B399DA0033D7EA00935A040160
:10832000B394D40093850A0013050A00336B9700B9
:10833000EF10D01A1309050093850A0013050A00EF
:10834000931B0401EF10101593DB0B019304050040
:108350009305050013850B00EF1010111319090187
:1083600013570B013367E900138A0400637EA700EB
:1083700033078700138AF4FF636887006376A700DA
:10838000138AE4FF33078700B304A74093850A00EC
:1083900013850400EF1090141309050093850A005B
:1083A00013850400EF10100F9304050093050500DA
:1083B00013850B00EF10500B13170B011357070118
:1083C00013190901B367E9001387040063FEA700CE
:1083D000B38787001387F4FF63E8870063F6A7007D
:1083E0001387E4FFB3878700131A0A01B384A740F9
:1083F000336AEA006FF0DFDF63ECD51EB7070100D8
:1084000063F4F6041307F00FB335D70093953500E6
:1084100033D7B60097870100938747EDB387E7000E
:1084200003C70700130A00023307B700330AEA4004
:1084300063160A0213041000E3E096E833B6CA009C
:10844000134416006FF05FE7B707000193050001C2
:10845000E3E0F6FC930580016FF09FFBB35CE60060
:10846000B3964601B3ECDC0033D4E40093DB0C019B
:10847000B397440133D7EA0093850B00130504003A
:10848000336BF700B3194601EF10500513090500CF
:1084900093850B0013050400139C0C01EF10807FE3
:1084A000135C0C01930405009305050013050C00F3
:1084B000EF10807B1319090113570B013367E90093
:1084C00013840400637EA700330797011384F4FF2D
:1084D000636897016376A7001384E4FF330797016D
:1084E000B304A74093850B0013850400EF10007FB1
:1084F0001309050093850B0013850400EF108079A4
:10850000930405009305050013050C00EF10C075DA
:1085100093170B011319090193D70701B367F900EA
:108520001386040063FEA700B38797011386F4FF48
:1085300063E8970163F6A7001386E4FFB38797010A
:1085400013140401B70B01003364C4001389FBFF4B
:10855000337D240133F92901B384A7409305090031
:1085600013050D00EF104070935C040193050900A2
:10857000130B050013850C00EF10006F93D9090150
:10858000130C05009385090013850C00EF10C06DD6
:10859000130905009385090013050D00EF10C06C49
:1085A0003305850193570B013385A700637485015B
:1085B0003309790193570501B387270163E6F40274
:1085C000E392F4BCB70701009387F7FF3375F5001A
:1085D00013150501337BFB0033964A013305650112
:1085E000130A0000E37AA6CC1304F4FF6FF09FB9DE
:1085F000130A0000130400006FF01FCC130101FBED
:108600002324810423229104232E31032322910366
:108610002326110423202105232C4103232A51035F
:108620002328610323267103232481032320A1032C
:10863000232EB101930C0500938905001304050056
:1086400093840500639E062613090600138A06001C
:10865000978A0100938A8AC963F4C514B707010099
:108660006376F6129307F00F63F4C700130A8000D5
:10867000B3574601B38AFA0003C70A001305000284
:1086800033074701330AE540630C0A00B3954901FB
:1086900033D7EC0033194601B364B70033944C016F
:1086A000935A090193850A0013850400EF100063B3
:1086B0009309050093850A00131B09011385040023
:1086C000EF10405D135B0B019305050013050B00D4
:1086D000EF1080599399090193570401B3E7F9000A
:1086E00063FAA700B387270163E6270163F4A700B5
:1086F000B3872701B384A74093850A00138504003C
:10870000EF10C05D9309050093850A0013850400EE
:10871000EF104058131404019305050093990901C3
:1087200013050B0013540401EF10005433E48900C7
:10873000637AA40033042401636624016374A400F3
:10874000330424013304A44033554401930500004D
:108750008320C104032481048324410403290104E8
:108760008329C103032A8103832A4103032B0103C5
:10877000832BC102032C8102832C4102032D0102B1
:10878000832DC1011301010567800000B7070001B7
:10879000130A0001E36EF6EC130A80016FF05FED3F
:1087A000631A06009305000013051000EF10804EB9
:1087B00013090500B7070100637AF90E9307F00F5C
:1087C00063F42701130A8000B3574901B38AFA0002
:1087D00003C70A0013050002B38429413307470188
:1087E000330AE540E30E0AEA33194901B3DAE90036
:1087F000B395490133D7EC0093540901336BB700AB
:1088000013850A0093850400EF10404D930905007D
:1088100093850400931B090113850A00EF1080471C
:1088200093DB0B019305050013850B00EF10C0438C
:108830009399090193570B01B3E7F90033944C0165
:1088400063FAA700B387270163E6270163F4A70053
:10885000B3872701B38AA7409385040013850A00D4
:10886000EF10C047930905009385040013850A00A3
:10887000EF1040429305050013850B00EF10C03E3A
:1088800093150B019399090193D50501B3E5B9003F
:1088900063FAA500B385250163E6250163F4A5000D
:1088A000B3852501B384A5406FF09FDFB7070001B2
:1088B000130A0001E36AF9F0130A80016FF0DFF098
:1088C000E3E8D5E8B707010063FCF604930BF00F6B
:1088D00033B5DB001315350033D7A60097870100A9
:1088E0009387C7A0B387E70083CB070093050002F7
:1088F000B38BAB00338B7541631E0B0263E436010F
:1089000063EACC003384CC40B386D94033B58C00C5
:10891000B384A64013050400938504006FF05FE361
:10892000B707000113050001E3E8F6FA130580011B
:108930006FF09FFAB3966601335D7601336DDD000B
:1089400033D47901B395690133DC7C0193540D0173
:10895000336CBC001305040093850400B31A660150
:10896000EF10C037130A05009385040013050400B7
:1089700033996C01931C0D01EF10C03193DC0C0195
:10898000130405009305050013850C00EF10C02D9E
:10899000131A0A0113570C013367EA00130A040083
:1089A000637EA7003307A701130AF4FF6368A701DA
:1089B0006376A700130AE4FF3307A701B309A740B2
:1089C0009385040013850900EF104031938504005E
:1089D0001304050013850900EF10C02B9305050053
:1089E0009304050013850C00EF10002893150C016B
:1089F0001314040193D50501B365B4001387040073
:108A000063FEA500B385A5011387F4FF63E8A50104
:108A100063F6A5001387E4FFB385A501131A0A01C5
:108A2000B70C0100336AEA001384FCFFB3778A00B5
:108A300033F48A00B384A54013850700930504002E
:108A40002326F100135A0A01EF10002293090500B2
:108A50009305040013050A00EF10002113DC0A013E
:108A6000930D050093050C0013050A00EF10C01FBD
:108A70008327C100130A050093050C001385070026
:108A8000EF10801E3305B50113D709013307A70086
:108A90006374B701330A9A01B70701009387F7FFA0
:108AA000935507013377F70013170701B3F7F90060
:108AB000B3854501B307F70063E6B400639EB400D5
:108AC000637CF90033865741B3B7C700B385A5412E
:108AD000B385F54093070600B307F9403339F90031
:108AE000B385B440B385254133947501B3D767018D
:108AF0003365F400B3D565016FF09FC5B7078000FB
:108B0000130101FF9387F7FF33F7A70023248100A8
:108B100023202101135475011359F50113D5750153
:108B2000B3F7B7001374F40F1375F50F2326110074
:108B30002322910093D5F501131637009397370040
:108B40003307A440631EB9186358E00A631805068A
:108B5000639C07009307F00F630CF404930706006F
:108B6000130504006F00C00B1307F7FF631E070215
:108B7000B387C70013050400139757006352070A11
:108B8000130515001307F00F6304E5323707007E65
:108B900093F617001307F7FF93D71700B3F7E70013
:108BA000B3E7D7006F00C0079306F00F6310D4023D
:108BB000930706001305F00F6F0080069306F00F71
:108BC000E308D4FEB7060004B3E7D7009306B0016C
:108BD00063D6E600930710006FF09FF9930600023A
:108BE000B386E640B3D5E700B397D700B337F000BC
:108BF000B3E7F5006FF0DFF76304070863100404C0
:108C0000630006029306F0FF6316D700B387C70020
:108C10006FF09FF69306F00F1347F7FF631AD50224
:108C200013F777006308072813F7F700930640004F
:108C30006302D728938747006F00C0279306F00F81
:108C4000E300D5FEB70600043307E0403366D600E4
:108C50009306B00163D6E600130710006F00C00151
:108C600093060002B355E6003387E6403317E6006B
:108C70003337E00033E7E500B387E7006FF0DFEF5D
:108C8000130514009376F50F130710006340D70403
:108C90006318040213050000E30406F86386072046
:108CA000B387C70013975700E35C07F6370700FC4C
:108CB0001307F7FFB3F7E700130510006FF05FF637
:108CC000E30A06EE639407166FF09FEE1307F00FAA
:108CD0006300E51E3307F600935717006FF05FF44B
:108CE0006350E00863160504E38607E61307F7FF01
:108CF00063140702B307F6401305040013975700E7
:108D0000E35007F2B70400049384F4FFB3F4970030
:108D1000130405006F00C0139306F00FE30AD4E8B4
:108D20009306B00163D0E602930710006FF09FFC3A
:108D30009306F00FE30ED4E6B7060004B3E7D700BE
:108D40006FF01FFE93060002B3D5E7003387E640BD
:108D5000B397E700B337F000B3E7F5006FF09FF982
:108D6000630E0706631E040213890500E30A06EA80
:108D70009306F0FF6318D700B387C7401389050037
:108D80006FF0DFF79306F00F1347F7FFE30AD5E81C
:108D90009306B00163D4E602130710006F0080034E
:108DA0009306F00F13890500E30CD5E6B70600041F
:108DB0003307E0403366D6006FF09FFD9306000254
:108DC0003358E6003387E6403317E6003337E000D8
:108DD0003367E800B387E7406FF05FFA13071400CA
:108DE0001377F70F9306100063CAE604631C0402AE
:108DF00063180600639E0712130500006F008003CE
:108E0000638C07123307F64093165700B387C740A9
:108E100063C0061293070700631607069307000056
:108E20006FF09FFDE31006EA639C0710B70700028E
:108E30001305F00F130900006F00C007B304F640DC
:108E40001397540063540704B384C7401389050083
:108E500013850400EF00D06E1305B5FFB394A40092
:108E6000634A85023305854013051500130400028B
:108E7000B3D7A4003305A440B394A400B334900046
:108E8000B3E79700130500006FF09FD9E38804F85B
:108E90006FF01FFCB70700FC9387F7FF3305A44072
:108EA000B3F7F4006FF0DFD7930706006FF05FD7DA
:108EB0009307000013975700635E07001305150022
:108EC0001307F00F6302E508370700FC1307F7FFED
:108ED000B3F7E7001307F00F93D737006318E500E7
:108EE00063860700B70740001309000037078000BA
:108EF0001307F7FF1375F50FB3F7E70013177501A5
:108F0000370580808320C100032481001305F5FF0D
:108F100033F5A7001319F9013365E5003365250121
:108F2000832441000329010013010101678000002F
:108F3000138905006FF01FF5930706006FF09FF48B
:108F4000138905006FF01FC7930700006FF09FF8AB
:108F5000130101FD23229102232A5101935475012B
:108F6000B70A80002320210323286101938AFAFF96
:108F70002326110223248102232E3101232C4101B7
:108F8000232671012324810193F4F40F138B050030
:108F9000B3FAAA001359F501638804089307F00F88
:108FA0006384F40A939A3A00B7070004B3EAFA001C
:108FB000938414F8930B000013557B013704800051
:108FC0001304F4FF1375F50F33746401135BFB0195
:108FD000630C05089307F00F6308F50A13143400B7
:108FE000B70700043364F400130515F89307000075
:108FF00013972B003367F7001307F7FF9306E00082
:10900000B3496901338AA44063E0E60A9776010018
:1090100093864626131727003307D7000327070038
:109020003307D70067000700638A0A0213850A0026
:10903000EF0010519307B5FF9304A0F8B39AFA001C
:10904000B384A4406FF01FF79304F00F930B20003C
:10905000E3840AF6930B30006FF01FF693040000D0
:10906000930B10006FF05FF5630A04021305040010
:10907000EF00104D9307B5FF3314F4009307A0F8E9
:109080003385A7406FF09FF61305F00F930720007C
:10909000E30004F6930730006FF09FF5130500001E
:1090A000930710006FF0DFF4131B540063F68A126D
:1090B000130AFAFF13090000935B0B013704010048
:1090C00093850B001304F4FF13850A00EF00903C16
:1090D00033748B0093050500130C05001305040081
:1090E000EF0090389304050093850B0013850A0068
:1090F000EF00D03E13590901131505013365A9008E
:1091000013090C00637E9500330565011309FCFF0C
:1091100063686501637695001309ECFF330565010B
:10912000B304954093850B0013850400EF0090363F
:1091300093050500130C050013050400EF00D03261
:10914000930A050093850B0013850400EF00103986
:109150001315050113040C00637E550133056501E9
:109160001304FCFF63686501637655011304ECFF8B
:109170003305650113190901330555413369890028
:109180003335A0003364A9001307FA076350E00ADF
:1091900093777400638A07009377F4009306400086
:1091A0006384D700130444009317440063DA070074
:1091B000B70700F89387F7FF3374F40013070A0822
:1091C0009307E00F1354340063D2E70C130400003C
:1091D0001307F00F6F00800B1399FA0193DA1A004E
:1091E0006FF09FED9309090013840A0093870B0029
:1091F00013072000E38CE7FC130730006382E708C5
:1092000013071000E392E7F81304000013070000AF
:109210006F00C00793090B006FF09FFD37044000FB
:1092200093090000930730006FF09FFC9307100034
:10923000B387E7401307B001E348F7FC1305EA09D9
:10924000B357F4003314A4003334800033E48700B0
:1092500093777400638A07009377F4001307400044
:109260006384E7001304440093175400135434003C
:10927000E3DE07F813040000130710006F0000017D
:10928000370440001307F00F9309000037058000F2
:109290001305F5FF3374A400370580801305F5FF2F
:1092A0001377F70F3374A400131777011395F9019F
:1092B0003364E4003365A4008320C10203248102E7
:1092C00083244102032901028329C101032A810168
:1092D000832A4101032B0101832BC100032C810050
:1092E0001301010367800000370780001307F7FFB1
:1092F000935675013378A70013D675019357F5017E
:1093000093F6F60F1305F00F3377B7001376F60FC9
:1093100093D5F5016398A6001305E0FF630E0806D8
:10932000678000006318A6001305E0FF630E0706C0
:109330006780000063940606133518006314060066
:1093400063060704631C05006394B700635ED600E0
:10935000130510006396070067800000E39E05FE7A
:109360001305F0FF6780000063DAC6001305F0FF05
:10937000E38407FE1305100067800000E36A07FD21
:1093800013050000E364E8FE6FF01FFD1305000005
:10939000E30408FC6FF0DFFBE308D6F8E31606FAF7
:1093A000E30807FA6FF05FFA13351800E38C06F84C
:1093B0006FF09FF9370780001307F7FF9356750189
:1093C0003378A70013D675019357F50193F6F60F7E
:1093D0001305F00F3377B7001376F60F93D5F50129
:1093E0006398A60013052000630E0806678000003E
:1093F0006318A60013052000630E070667800000AF
:109400006394060613351800631406006306070408
:10941000631C05006394B700635ED600130510005B
:109420006396070067800000E39E05FE1305F0FFCA
:109430006780000063DAC6001305F0FFE38407FECF
:109440001305100067800000E36A07FD13050000A4
:10945000E364E8FE6FF01FFD13050000E30408FC61
:109460006FF0DFFBE308D6F8E31606FAE30807FA25
:109470006FF05FFA13351800E38C06F86FF09FF970
:10948000130101FD2322910223202103B704800050
:1094900013597501232E3101232671019384F4FFA2
:1094A0002326110223248102232C4101232A510166
:1094B0002328610123248101232291011379F90FCB
:1094C000938B0500B3F4A4009359F501630A0908CE
:1094D0009307F00F6306F90A93943400B70700046A
:1094E000B3E4F400130919F8130B000013D57B0142
:1094F000370480001304F4FF1375F50F33747401FF
:1095000093DBFB01630E05089307F00F630AF50A6E
:1095100013143400B70700043364F400130515F87E
:109520009306000093172B00B3E7D7003309A90077
:109530009387F7FF1307E00033CA7901930A1900F4
:109540006360F70A17770100130787D69397270000
:10955000B387E70083A70700B387E70067800700AA
:10956000638A040213850400EF00807D9307B5FF32
:109570001309A0F8B394F4003309A9406FF0DFF6A3
:109580001309F00F130B2000E38204F6130B3000D5
:109590006FF0DFF513090000130B10006FF01FF5DB
:1095A000630A040213050400EF0080799307B5FFF6
:1095B0003314F4009307A0F83385A7406FF05FF6EB
:1095C0001305F00F93062000E30E04F49306300019
:1095D0006FF05FF513050000930610006FF09FF425
:1095E000370C0100130BFCFF93DB0401935C0401B7
:1095F000B3F464013374640193050400138504001B
:10960000EF008066930504009309050013850B00A5
:10961000EF0080651304050093850C0013850B0093
:10962000EF008064930B05009385040013850C0004
:10963000EF0080633305850093D709013385A700C8
:1096400063748500B38B8B01B37765019397070132
:10965000B3F96901B387370113946700333480008D
:1096600093D7A70113550501B367F40033047501BF
:10967000131464003364F4009317440063D6070E98
:10968000935714001374140033E487001387FA0708
:109690006350E00E93777400638A07009377F400B9
:1096A000930640006384D7001304440093174400DA
:1096B00063DA0700B70700F89387F7FF3374F40005
:1096C00013870A089307E00F63C4E7109357340029
:1096D0006F000003138A09001384040093060B0033
:1096E000930720006386F60E93073000638AF60C1A
:1096F000130610009307000013070000E398C6F854
:10970000370480001304F4FF37058080B3F7870027
:109710001305F5FF8320C102032481021377F70F9D
:10972000B3F7A700131777011315FA01B3E7E700A2
:1097300083244102032901028329C101032A8101F3
:10974000832A4101032B0101832BC100032C8100DB
:10975000832C410033E5A70013010103678000005B
:10976000138A0B006FF0DFF7930A09006FF01FF206
:1097700093071000B387E7401307B0016340F70673
:10978000938AEA09B357F400331454013334800048
:1097900033E4870093777400638A07009377F400BB
:1097A000130740006384E700130444009317540038
:1097B00063CA070293573400130700006FF05FF489
:1097C000B70740001307F00F130A00006FF05FF3B4
:1097D000930700001307F00F6FF09FF2930700004C
:1097E0006FF09FFD93070000130710006FF05FF10B
:1097F000B70780009387F7FF130101FF33F7A70036
:109800009356750113D67501B3F7B7002322910063
:109810002320210193F6F60F131837001376F60F65
:1098200023261100232481001307F00F9354F50120
:10983000138906001305060093D5F50193973700A9
:109840006314E6006394070093C515003387C64090
:10985000639A951A6356E00A63160606639C07002E
:109860009307F00F638CF604930708001385060036
:109870006F00C0141307F7FF631E0702B3870701C9
:109880001385060013975700635A07121305150036
:109890001307F00F630EE5323707007E93F61700CB
:1098A0001307F7FF93D71700B3F7E700B3E7D70025
:1098B0006F00C0101306F00F639EC60093070800E8
:1098C0006F0040071306F00FE38AC6FE3706000458
:1098D000B3E7C7001306B0016356E6009307100014
:1098E0006FF0DFF9130600023306E640B3D5E70058
:1098F000B397C700B337F000B3E7F5006FF01FF878
:1099000063000708639C0602631808001307F00F42
:109910006316E60A6F0000029306F0FF6316D70095
:10992000B38707016FF01FF69306F00F1347F7FF99
:109930006310D6021305F00F6F0040089306F00F76
:10994000E30AD6FEB70600043307E0403368D800C8
:109950009306B00163D6E600130710006F00C00144
:10996000930600023356E8003387E6403317E800D9
:109970003337E0003367E600B387E7006FF09FF00E
:10998000138516001376F50F130710006342C70600
:10999000639406041305000063020802638607222D
:1099A000B387070113975700635A0700370700FC76
:1099B0001307F7FFB3F7E7001305100013F777005D
:1099C000630A072013F7F700930640006304D720CB
:1099D000938747006F000020E30E08F4E38007EE52
:1099E000B70700021305F00F930400006F00801EFC
:1099F0001307F00F630EE51C3307F80093571700A9
:109A00006FF0DFFB6350E00863160604E38A07E4A7
:109A10001307F7FF63140702B307F8401385060026
:109A200013975700E35C07F8370400041304F4FFAE
:109A300033F48700130905006F0080131306F00F3D
:109A4000E38EC6E61306B0016350E60293071000EA
:109A50006FF09FFC1306F00FE382C6E637060004A2
:109A6000B3E7C7006FF01FFE13060002B3D5E7008F
:109A70003307E640B397E700B337F000B3E7F500EC
:109A80006FF09FF963020708639E060263180800DF
:109A90001307F00F938405006FF09FE79306F0FF24
:109AA0006318D700B3870741938405006FF05FF711
:109AB0009306F00F1347F7FF6310D6029384050057
:109AC0006FF05FE79306F00FE30AD6FEB7060004D7
:109AD0003307E0403368D8009306B00163D6E60050
:109AE000130710006F00C001930600023356E80010
:109AF0003387E6403317E8003337E0003367E6008A
:109B0000B387E7406FF05FFA138716001377F70FFC
:109B1000130610006344E604639C06026318080001
:109B200063980712130500006FF01FEC638607129D
:109B30003307F84093165700B387074163CA0610EE
:109B40009307070063100706930700006FF09FFD5F
:109B5000E31608E8E39407F66FF09FE83304F84053
:109B6000131754006354070433840741938405009A
:109B700013050400EF00C01C1305B5FF3314A40047
:109B8000634A250333052541130515001307000219
:109B9000B357A4003305A7403314A4003334800026
:109BA000B3E78700130500006FF05FE1E30E04F8F0
:109BB0006FF01FFCB70700FC9387F7FF3305A94040
:109BC000B377F4006FF09FDF930708006FF01FDF9B
:109BD0009307000013975700635E070013051500F5
:109BE0001307F00F630EE506370700FC1307F7FFB6
:109BF000B3F7E7001307F00F93D737006318E500BA
:109C000063860700B7074000930400003707800011
:109C10001307F7FF1375F50FB3F7E7001317750177
:109C2000370580808320C100032481001305F5FFE0
:109C300033F5A7009394F4013365E500336595008F
:109C40000329010083244100130101016780000002
:109C5000938405006FF01FF5930708006FF09FF4E1
:109C6000930700006FF01FF91306050013050000AD
:109C700093F61500638406003305C50093D51500DF
:109C800013161600E39605FE678000006340050684
:109C900063C6050613860500930505001305F0FF4E
:109CA000630C060293061000637AB6006358C00086
:109CB0001316160093961600E36AB6FE130500000D
:109CC00063E6C500B385C5403365D50093D616005D
:109CD00013561600E39606FE67800000938200008C
:109CE000EFF05FFB13850500678002003305A0409D
:109CF00063D80500B305B0406FF0DFF9B305B0409D
:109D000093820000EFF01FF93305A0406780020046
:109D10009382000063CA0500634C0500EFF09FF7D3
:109D20001385050067800200B305B040E35805FEC7
:109D30003305A040EFF01FF63305B0406780020006
:109D4000B7070100637AF5029307F00FB3B7A700D6
:109D500093973700130700023307F740B357F50016
:109D60001765010013058558B307F50003C5070003
:109D70003305A74067800000370700019307000103
:0C9D8000E36AE5FC930780016FF0DFFC54
:02000004800278
:1000000049444C4500000000244BFEFFBC4AFEFF63
:10001000D84AFEFFF04AFEFF004BFEFFF44CFEFF05
:100020008C4CFEFFA84CFEFFC04CFEFFD04CFEFFE8
:10003000546D7220537663001C56FEFF1C56FEFF63
:100040001C56FEFF0457FEFFAC56FEFFF456FEFFA3
:100050001C56FEFF1C56FEFF0457FEFFAC56FEFF6B
:10006000546D725100000000286E756C6C29000000
:10007000406DFEFF7C70FEFF6870FEFF7C70FEFF2F
:100080007C70FEFF7C70FEFF7C70FEFFEC6DFEFF5F
:100090007C70FEFF7C70FEFF846DFEFF046EFEFF31
:1000A0007C70FEFF906DFEFF9C6DFEFF9C6DFEFF61
:1000B0009C6DFEFF9C6DFEFF9C6DFEFF9C6DFEFF28
:1000C0009C6DFEFF9C6DFEFF9C6DFEFF7C70FEFF35
:1000D0007C70FEFF7C70FEFF7C70FEFF7C70FEFF7C
:1000E0007C70FEFF7C70FEFF7C70FEFF7C70FEFF6C
:1000F0007C70FEFF7C70FEFF7C70FEFF7C70FEFF5C
:100100007C70FEFF7C70FEFF7C70FEFF7C70FEFF4B
:100110007C70FEFF7C70FEFF7C70FEFF7C70FEFF3B
:100120007C70FEFF7C70FEFF7C70FEFF7C70FEFF2B
:100130007C70FEFF7C70FEFF7C70FEFF7C70FEFF1B
:100140007C70FEFF7C70FEFF7C70FEFF7C70FEFF0B
:100150007C70FEFF7C70FEFF7C70FEFF7C70FEFFFB
:100160007C70FEFF7C70FEFF7C70FEFF7C70FEFFEB
:10017000446EFEFF5C6FFEFF7C70FEFF7C70FEFF36
:100180007C70FEFF7C70FEFF7C70FEFF7C70FEFFCB
:100190007C70FEFF346EFEFF7C70FEFF7C70FEFF05
:1001A000EC6FFEFFF86FFEFF7C70FEFF7C70FEFFC1
:1001B000686EFEFF7C70FEFFE06FFEFF7C70FEFF4E
:1001C0007C70FEFF2070FEFF6D69616F750A000094
:1001D0006D69616F75320A0068756E6772790A0021
:1001E0004572726F7220696E2073705F666C6F70FB
:1001F00073207461736B73200D0A0000436865639C
:100200006B54696D657200004D61746831000000C7
:100210004D617468320000004D6174683300000065
:100220004D617468340000004D6174683500000051
:100230004D617468360000004D617468370000003D
:100240004D61746838000000D5E9F642DD9A124528
:10025000358E65C46F12833AA4B0C2C366E4FD460E
:10026000A30100C00000B0406F1283BACFF7414134
:100270005C8FFEFF988FFEFFA48FFEFF988FFEFF1E
:100280001090FEFF988FFEFFA48FFEFF5C8FFEFF95
:100290005C8FFEFF1090FEFFA48FFEFF748FFEFFA9
:1002A000748FFEFF748FFEFFAC8FFEFF3494FEFF51
:1002B0003494FEFFB494FEFF2C94FEFF2C94FEFFBA
:1002C0001495FEFFB494FEFF2C94FEFF1495FEFFE0
:1002D0002C94FEFFB494FEFF2894FEFF2894FEFFAA
:1002E0002894FEFF1495FEFF00010202030303039E
:1002F00004040404040404040505050505050505B6
:100300000505050505050505060606060606060695
:10031000060606060606060606060606060606067D
:100320000606060606060606070707070707070765
:10033000070707070707070707070707070707074D
:10034000070707070707070707070707070707073D
:10035000070707070707070707070707070707072D
:100360000707070707070707080808080808080815
:1003700008080808080808080808080808080808FD
:1003800008080808080808080808080808080808ED
:1003900008080808080808080808080808080808DD
:1003A00008080808080808080808080808080808CD
:1003B00008080808080808080808080808080808BD
:1003C00008080808080808080808080808080808AD
:1003D000080808080808080808080808080808089D
:0803E0000808080808080808D5
:1003E8001000000000000000017A5200017C0101A9
:1003F8001B0D02004C000000180000001C7CFEFFD2
:10040800DC05000000440E307089039507810188DF
:100418000292049305940696089709980A990B9AEC
:100428000C0370020AC144C844C944D244D344D41A
:1004380044D544D644D744D844D944DA440E004479
:100448000B0000005000000068000000A881FEFFBB
:100458000005000000440E50748802890393059932
:100468000B810192049406950796089709980A9AB1
:100478000C9B0D0320010AC144C844C944D244D38B
:1004880044D444D544D644D744D844D944DA44DB88
:08049800440E00440B000000BB
:1004AC00AAAAAAAA08000000FC8F010009000000FB
:040000058000004037
:00000001FF
